 alm_sys_select

 Timestamp is 614c7ffb (Thu Sep 23 13:24:11 2021)

 Preferred load address is 10000000

 Start         Length     Name                   Class
 0001:00000000 00000081H .text$di                CODE
 0001:00000090 0000237aH .text$mn                CODE
 0001:00002410 00000334H .text$x                 CODE
 0001:00002750 0000003bH .text$yd                CODE
 0002:00000000 00000548H .idata$5                DATA
 0002:00000548 00000004H .CRT$XCA                DATA
 0002:0000054c 0000000cH .CRT$XCU                DATA
 0002:00000558 00000004H .CRT$XCZ                DATA
 0002:0000055c 00000004H .CRT$XIA                DATA
 0002:00000560 00000004H .CRT$XIAA               DATA
 0002:00000564 00000004H .CRT$XIC                DATA
 0002:00000568 00000004H .CRT$XIZ                DATA
 0002:00000570 00000c10H .rdata                  DATA
 0002:00001180 00000640H .rdata$r                DATA
 0002:000017c0 00000004H .rtc$IAA                DATA
 0002:000017c4 00000004H .rtc$IZZ                DATA
 0002:000017c8 00000004H .rtc$TAA                DATA
 0002:000017cc 00000004H .rtc$TZZ                DATA
 0002:000017d0 000003d4H .xdata$x                DATA
 0002:00001bb0 00000530H .edata                  DATA
 0002:000020e0 0000003cH .idata$2                DATA
 0002:0000211c 00000014H .idata$3                DATA
 0002:00002130 00000548H .idata$4                DATA
 0002:00002678 00003388H .idata$6                DATA
 0003:00000000 00000014H .data                   DATA
 0003:00000014 000001e8H .data$r                 DATA
 0003:00000200 0000036cH .bss                    DATA
 0004:00000000 000000a0H .rsrc$01                DATA
 0004:000000a0 00000620H .rsrc$02                DATA

  Address         Publics by Value              Rva+Base       Lib:Object

 0000:00000000       ___safe_se_handler_table   00000000     <absolute>
 0000:00000000       ___safe_se_handler_count   00000000     <absolute>
 0000:00000000       ___guard_fids_table        00000000     <absolute>
 0000:00000000       ___guard_fids_count        00000000     <absolute>
 0000:00000000       ___guard_flags             00000000     <absolute>
 0000:00000000       ___ImageBase               10000000     <linker-defined>
 0001:00000090       ??0CAlm_sys_select@@QAE@PAVQWidget@@PBD@Z 10001090 f   alm_sys_select.obj
 0001:00000200       ??1CAlm_sys_select@@UAE@XZ 10001200 f i alm_sys_select.obj
 0001:00000260       ??4CAlm_sys_select@@QAEAAV0@ABV0@@Z 10001260 f i alm_sys_select.obj
 0001:000002b0       ??_ECAlm_sys_select@@UAEPAXI@Z 100012b0 f i alm_sys_select.obj
 0001:00000363       ??_ECAlm_sys_select@@WCI@AEPAXI@Z 10001363 f i alm_sys_select.obj
 0001:00000370       ?getSystemName@CAlm_sys_select@@QAE?AVQString@@XZ 10001370 f   alm_sys_select.obj
 0001:00000480       ?metaObject@CAlm_sys_select@@UBEPAVQMetaObject@@XZ 10001480 f i alm_sys_select.obj
 0001:00000490       ?qObject@CAlm_sys_select@@QAEPAVQObject@@XZ 10001490 f i alm_sys_select.obj
 0001:000004a0       ?selectSystem@CAlm_sys_select@@IAEXXZ 100014a0 f   alm_sys_select.obj
 0001:00000680       ?setSystem@CAlm_sys_select@@QAEXABVQString@@@Z 10001680 f   alm_sys_select.obj
 0001:00000690       ?setSystemNames@CAlm_sys_select@@QAE_NVQString@@@Z 10001690 f   alm_sys_select.obj
 0001:000009b0       _DllMain@12                100019b0 f   alm_sys_select.obj
 0001:000009c0       ?className@sys_selectBase@@UBEPBDXZ 100019c0 f   moc_sys_select.obj
 0001:000009d0       ?qt_cast@sys_selectBase@@UAEPAXPBD@Z 100019d0 f   moc_sys_select.obj
 0001:00000a30       ?qt_emit@sys_selectBase@@UAE_NHPAUQUObject@@@Z 10001a30 f   moc_sys_select.obj
 0001:00000a40       ?qt_invoke@sys_selectBase@@UAE_NHPAUQUObject@@@Z 10001a40 f   moc_sys_select.obj
 0001:00000ad0       ?qt_property@sys_selectBase@@UAE_NHHPAVQVariant@@@Z 10001ad0 f   moc_sys_select.obj
 0001:00000ae0       ?staticMetaObject@sys_selectBase@@SAPAVQMetaObject@@XZ 10001ae0 f   moc_sys_select.obj
 0001:00000b30       ?tr@sys_selectBase@@SA?AVQString@@PBD0@Z 10001b30 f   moc_sys_select.obj
 0001:00000b80       ??0sys_selectBase@@QAE@PAVQWidget@@PBDI@Z 10001b80 f   sys_select.obj
 0001:00000f20       ??_EQHBoxLayout@@WCI@AEPAXI@Z 10001f20 f i sys_select.obj
 0001:00000f28       ??_EQLabel@@WCI@AEPAXI@Z   10001f28 f i sys_select.obj
 0001:00000f30       ??_EQPushButton@@WCI@AEPAXI@Z 10001f30 f i sys_select.obj
 0001:00000f38       ??_EQVBoxLayout@@WCI@AEPAXI@Z 10001f38 f i sys_select.obj
 0001:00000f40       ??_Esys_selectBase@@WCI@AEPAXI@Z 10001f40 f i sys_select.obj
 0001:00000f50       ??_GQHBoxLayout@@UAEPAXI@Z 10001f50 f i sys_select.obj
 0001:00000f50       ??_EQHBoxLayout@@UAEPAXI@Z 10001f50 f i sys_select.obj
 0001:00000f80       ??_EQLabel@@UAEPAXI@Z      10001f80 f i sys_select.obj
 0001:00000f80       ??_GQLabel@@UAEPAXI@Z      10001f80 f i sys_select.obj
 0001:00000fb0       ??_GQPushButton@@UAEPAXI@Z 10001fb0 f i sys_select.obj
 0001:00000fb0       ??_EQPushButton@@UAEPAXI@Z 10001fb0 f i sys_select.obj
 0001:00000fe0       ??_GQSpacerItem@@UAEPAXI@Z 10001fe0 f i sys_select.obj
 0001:00000fe0       ??_EQSpacerItem@@UAEPAXI@Z 10001fe0 f i sys_select.obj
 0001:00001010       ??_EQVBoxLayout@@UAEPAXI@Z 10002010 f i sys_select.obj
 0001:00001010       ??_GQVBoxLayout@@UAEPAXI@Z 10002010 f i sys_select.obj
 0001:00001040       ??_Esys_selectBase@@UAEPAXI@Z 10002040 f i sys_select.obj
 0001:00001040       ??_Gsys_selectBase@@UAEPAXI@Z 10002040 f i sys_select.obj
 0001:00001070       ?languageChange@sys_selectBase@@MAEXXZ 10002070 f   sys_select.obj
 0001:00001180       ?metaObject@sys_selectBase@@UBEPAVQMetaObject@@XZ 10002180 f i sys_select.obj
 0001:00001190       ?className@CAlm_sys_select@@UBEPBDXZ 10002190 f   moc_alm_sys_select.obj
 0001:000011a0       ?qt_cast@CAlm_sys_select@@UAEPAXPBD@Z 100021a0 f   moc_alm_sys_select.obj
 0001:00001200       ?qt_emit@CAlm_sys_select@@UAE_NHPAUQUObject@@@Z 10002200 f   moc_alm_sys_select.obj
 0001:000012a0       ?qt_invoke@CAlm_sys_select@@UAE_NHPAUQUObject@@@Z 100022a0 f   moc_alm_sys_select.obj
 0001:000012e0       ?qt_property@CAlm_sys_select@@UAE_NHHPAVQVariant@@@Z 100022e0 f   moc_alm_sys_select.obj
 0001:000012f0       ?qt_static_property@CAlm_sys_select@@SA_NPAVQObject@@HHPAVQVariant@@@Z 100022f0 f   moc_alm_sys_select.obj
 0001:00001300       ?staticMetaObject@CAlm_sys_select@@SAPAVQMetaObject@@XZ 10002300 f   moc_alm_sys_select.obj
 0001:00001390       ?sysChanged@CAlm_sys_select@@IAEXABVQString@@@Z 10002390 f   moc_alm_sys_select.obj
 0001:00001400       ?tr@CAlm_sys_select@@SA?AVQString@@PBD0@Z 10002400 f   moc_alm_sys_select.obj
 0001:00001450       ?trUtf8@CAlm_sys_select@@SA?AVQString@@PBD0@Z 10002450 f   moc_alm_sys_select.obj
 0001:0000149c       ?adjustSize@QWidget@@UAEXXZ 1000249c f   qt-mt323:qt-mt323.dll
 0001:000014a2       ?checkConnectArgs@QObject@@MAE_NPBDPBV1@0@Z 100024a2 f   qt-mt323:qt-mt323.dll
 0001:000014a8       ?childEvent@QObject@@MAEXPAVQChildEvent@@@Z 100024a8 f   qt-mt323:qt-mt323.dll
 0001:000014ae       ?close@QWidget@@UAE_N_N@Z  100024ae f   qt-mt323:qt-mt323.dll
 0001:000014b4       ?closeEvent@QWidget@@MAEXPAVQCloseEvent@@@Z 100024b4 f   qt-mt323:qt-mt323.dll
 0001:000014ba       ?cmd@QPaintDevice@@MAE_NHPAVQPainter@@PATQPDevCmdParam@@@Z 100024ba f   qt-mt323:qt-mt323.dll
 0001:000014c0       ?connectNotify@QObject@@MAEXPBD@Z 100024c0 f   qt-mt323:qt-mt323.dll
 0001:000014c6       ?contextMenuEvent@QWidget@@MAEXPAVQContextMenuEvent@@@Z 100024c6 f   qt-mt323:qt-mt323.dll
 0001:000014cc       ?create@QWidget@@MAEXPAUHWND__@@_N1@Z 100024cc f   qt-mt323:qt-mt323.dll
 0001:000014d2       ?customEvent@QObject@@MAEXPAVQCustomEvent@@@Z 100024d2 f   qt-mt323:qt-mt323.dll
 0001:000014d8       ?customWhatsThis@QWidget@@UBE_NXZ 100024d8 f   qt-mt323:qt-mt323.dll
 0001:000014de       ?destroy@QWidget@@MAEX_N0@Z 100024de f   qt-mt323:qt-mt323.dll
 0001:000014e4       ?disconnectNotify@QObject@@MAEXPBD@Z 100024e4 f   qt-mt323:qt-mt323.dll
 0001:000014ea       ?dragEnterEvent@QWidget@@MAEXPAVQDragEnterEvent@@@Z 100024ea f   qt-mt323:qt-mt323.dll
 0001:000014f0       ?dragLeaveEvent@QWidget@@MAEXPAVQDragLeaveEvent@@@Z 100024f0 f   qt-mt323:qt-mt323.dll
 0001:000014f6       ?dragMoveEvent@QWidget@@MAEXPAVQDragMoveEvent@@@Z 100024f6 f   qt-mt323:qt-mt323.dll
 0001:000014fc       ?drawContents@QFrame@@MAEXPAVQPainter@@@Z 100024fc f   qt-mt323:qt-mt323.dll
 0001:00001502       ?drawFrame@QFrame@@MAEXPAVQPainter@@@Z 10002502 f   qt-mt323:qt-mt323.dll
 0001:00001508       ?dropEvent@QWidget@@MAEXPAVQDropEvent@@@Z 10002508 f   qt-mt323:qt-mt323.dll
 0001:0000150e       ?enabledChange@QWidget@@MAEX_N@Z 1000250e f   qt-mt323:qt-mt323.dll
 0001:00001514       ?enterEvent@QWidget@@MAEXPAVQEvent@@@Z 10002514 f   qt-mt323:qt-mt323.dll
 0001:0000151a       ?event@QWidget@@MAE_NPAVQEvent@@@Z 1000251a f   qt-mt323:qt-mt323.dll
 0001:00001520       ?eventFilter@QObject@@UAE_NPAV1@PAVQEvent@@@Z 10002520 f   qt-mt323:qt-mt323.dll
 0001:00001526       ?focusInEvent@QWidget@@MAEXPAVQFocusEvent@@@Z 10002526 f   qt-mt323:qt-mt323.dll
 0001:0000152c       ?focusNextPrevChild@QWidget@@MAE_N_N@Z 1000252c f   qt-mt323:qt-mt323.dll
 0001:00001532       ?focusOutEvent@QWidget@@MAEXPAVQFocusEvent@@@Z 10002532 f   qt-mt323:qt-mt323.dll
 0001:00001538       ?fontChange@QWidget@@MAEXABVQFont@@@Z 10002538 f   qt-mt323:qt-mt323.dll
 0001:0000153e       ?fontInf@QPaintDevice@@MBEHPAVQFont@@H@Z 1000253e f   qt-mt323:qt-mt323.dll
 0001:00001544       ?fontMet@QPaintDevice@@MBEHPAVQFont@@HPBDH@Z 10002544 f   qt-mt323:qt-mt323.dll
 0001:0000154a       ?frameChanged@QHBox@@MAEXXZ 1000254a f   qt-mt323:qt-mt323.dll
 0001:00001550       ?handle@QPaintDevice@@UBEPAUHDC__@@XZ 10002550 f   qt-mt323:qt-mt323.dll
 0001:00001556       ?heightForWidth@QWidget@@UBEHH@Z 10002556 f   qt-mt323:qt-mt323.dll
 0001:0000155c       ?hide@QWidget@@UAEXXZ      1000255c f   qt-mt323:qt-mt323.dll
 0001:00001562       ?hideEvent@QWidget@@MAEXPAVQHideEvent@@@Z 10002562 f   qt-mt323:qt-mt323.dll
 0001:00001568       ?imComposeEvent@QWidget@@MAEXPAVQIMEvent@@@Z 10002568 f   qt-mt323:qt-mt323.dll
 0001:0000156e       ?imEndEvent@QWidget@@MAEXPAVQIMEvent@@@Z 1000256e f   qt-mt323:qt-mt323.dll
 0001:00001574       ?imStartEvent@QWidget@@MAEXPAVQIMEvent@@@Z 10002574 f   qt-mt323:qt-mt323.dll
 0001:0000157a       ?insertChild@QObject@@UAEXPAV1@@Z 1000257a f   qt-mt323:qt-mt323.dll
 0001:00001580       ?keyPressEvent@QWidget@@MAEXPAVQKeyEvent@@@Z 10002580 f   qt-mt323:qt-mt323.dll
 0001:00001586       ?keyReleaseEvent@QWidget@@MAEXPAVQKeyEvent@@@Z 10002586 f   qt-mt323:qt-mt323.dll
 0001:0000158c       ?leaveEvent@QWidget@@MAEXPAVQEvent@@@Z 1000258c f   qt-mt323:qt-mt323.dll
 0001:00001592       ?metric@QWidget@@MBEHH@Z   10002592 f   qt-mt323:qt-mt323.dll
 0001:00001598       ?minimumSizeHint@QWidget@@UBE?AVQSize@@XZ 10002598 f   qt-mt323:qt-mt323.dll
 0001:0000159e       ?mouseDoubleClickEvent@QWidget@@MAEXPAVQMouseEvent@@@Z 1000259e f   qt-mt323:qt-mt323.dll
 0001:000015a4       ?mouseMoveEvent@QWidget@@MAEXPAVQMouseEvent@@@Z 100025a4 f   qt-mt323:qt-mt323.dll
 0001:000015aa       ?mousePressEvent@QWidget@@MAEXPAVQMouseEvent@@@Z 100025aa f   qt-mt323:qt-mt323.dll
 0001:000015b0       ?mouseReleaseEvent@QWidget@@MAEXPAVQMouseEvent@@@Z 100025b0 f   qt-mt323:qt-mt323.dll
 0001:000015b6       ?move@QWidget@@UAEXHH@Z    100025b6 f   qt-mt323:qt-mt323.dll
 0001:000015bc       ?moveEvent@QWidget@@MAEXPAVQMoveEvent@@@Z 100025bc f   qt-mt323:qt-mt323.dll
 0001:000015c2       ?paintEvent@QFrame@@MAEXPAVQPaintEvent@@@Z 100025c2 f   qt-mt323:qt-mt323.dll
 0001:000015c8       ?paletteChange@QWidget@@MAEXABVQPalette@@@Z 100025c8 f   qt-mt323:qt-mt323.dll
 0001:000015ce       ?polish@QWidget@@UAEXXZ    100025ce f   qt-mt323:qt-mt323.dll
 0001:000015d4       ?property@QObject@@UBE?AVQVariant@@PBD@Z 100025d4 f   qt-mt323:qt-mt323.dll
 0001:000015da       ?removeChild@QObject@@UAEXPAV1@@Z 100025da f   qt-mt323:qt-mt323.dll
 0001:000015e0       ?reparent@QWidget@@UAEXPAV1@IABVQPoint@@_N@Z 100025e0 f   qt-mt323:qt-mt323.dll
 0001:000015e6       ?resize@QWidget@@UAEXHH@Z  100025e6 f   qt-mt323:qt-mt323.dll
 0001:000015ec       ?resizeEvent@QFrame@@MAEXPAVQResizeEvent@@@Z 100025ec f   qt-mt323:qt-mt323.dll
 0001:000015f2       ?resolution@QPaintDevice@@UBEHXZ 100025f2 f   qt-mt323:qt-mt323.dll
 0001:000015f8       ?setAcceptDrops@QWidget@@UAEX_N@Z 100025f8 f   qt-mt323:qt-mt323.dll
 0001:000015fe       ?setActiveWindow@QWidget@@UAEXXZ 100025fe f   qt-mt323:qt-mt323.dll
 0001:00001604       ?setAutoMask@QWidget@@UAEX_N@Z 10002604 f   qt-mt323:qt-mt323.dll
 0001:0000160a       ?setBackgroundColor@QWidget@@UAEXABVQColor@@@Z 1000260a f   qt-mt323:qt-mt323.dll
 0001:00001610       ?setBackgroundMode@QWidget@@UAEXW4BackgroundMode@Qt@@@Z 10002610 f   qt-mt323:qt-mt323.dll
 0001:00001616       ?setBackgroundOrigin@QWidget@@UAEXW4BackgroundOrigin@1@@Z 10002616 f   qt-mt323:qt-mt323.dll
 0001:0000161c       ?setBackgroundPixmap@QWidget@@UAEXABVQPixmap@@@Z 1000261c f   qt-mt323:qt-mt323.dll
 0001:00001622       ?setCaption@QWidget@@UAEXABVQString@@@Z 10002622 f   qt-mt323:qt-mt323.dll
 0001:00001628       ?setCursor@QWidget@@UAEXABVQCursor@@@Z 10002628 f   qt-mt323:qt-mt323.dll
 0001:0000162e       ?setEnabled@QWidget@@UAEX_N@Z 1000262e f   qt-mt323:qt-mt323.dll
 0001:00001634       ?setEraseColor@QWidget@@UAEXABVQColor@@@Z 10002634 f   qt-mt323:qt-mt323.dll
 0001:0000163a       ?setErasePixmap@QWidget@@UAEXABVQPixmap@@@Z 1000263a f   qt-mt323:qt-mt323.dll
 0001:00001640       ?setFocus@QWidget@@UAEXXZ  10002640 f   qt-mt323:qt-mt323.dll
 0001:00001646       ?setFocusPolicy@QWidget@@UAEXW4FocusPolicy@1@@Z 10002646 f   qt-mt323:qt-mt323.dll
 0001:0000164c       ?setFocusProxy@QWidget@@UAEXPAV1@@Z 1000264c f   qt-mt323:qt-mt323.dll
 0001:00001652       ?setFont@QWidget@@UAEXABVQFont@@@Z 10002652 f   qt-mt323:qt-mt323.dll
 0001:00001658       ?setFrameRect@QFrame@@UAEXABVQRect@@@Z 10002658 f   qt-mt323:qt-mt323.dll
 0001:0000165e       ?setFrameStyle@QFrame@@UAEXH@Z 1000265e f   qt-mt323:qt-mt323.dll
 0001:00001664       ?setGeometry@QWidget@@UAEXABVQRect@@@Z 10002664 f   qt-mt323:qt-mt323.dll
 0001:0000166a       ?setGeometry@QWidget@@UAEXHHHH@Z 1000266a f   qt-mt323:qt-mt323.dll
 0001:00001670       ?setIcon@QWidget@@UAEXABVQPixmap@@@Z 10002670 f   qt-mt323:qt-mt323.dll
 0001:00001676       ?setIconText@QWidget@@UAEXABVQString@@@Z 10002676 f   qt-mt323:qt-mt323.dll
 0001:0000167c       ?setKeyCompression@QWidget@@MAEX_N@Z 1000267c f   qt-mt323:qt-mt323.dll
 0001:00001682       ?setLineWidth@QFrame@@UAEXH@Z 10002682 f   qt-mt323:qt-mt323.dll
 0001:00001688       ?setMargin@QFrame@@UAEXH@Z 10002688 f   qt-mt323:qt-mt323.dll
 0001:0000168e       ?setMask@QWidget@@UAEXABVQBitmap@@@Z 1000268e f   qt-mt323:qt-mt323.dll
 0001:00001694       ?setMask@QWidget@@UAEXABVQRegion@@@Z 10002694 f   qt-mt323:qt-mt323.dll
 0001:0000169a       ?setMaximumSize@QWidget@@UAEXHH@Z 1000269a f   qt-mt323:qt-mt323.dll
 0001:000016a0       ?setMicroFocusHint@QWidget@@MAEXHHHH_NPAVQFont@@@Z 100026a0 f   qt-mt323:qt-mt323.dll
 0001:000016a6       ?setMidLineWidth@QFrame@@UAEXH@Z 100026a6 f   qt-mt323:qt-mt323.dll
 0001:000016ac       ?setMinimumSize@QWidget@@UAEXHH@Z 100026ac f   qt-mt323:qt-mt323.dll
 0001:000016b2       ?setMouseTracking@QWidget@@UAEX_N@Z 100026b2 f   qt-mt323:qt-mt323.dll
 0001:000016b8       ?setName@QWidget@@UAEXPBD@Z 100026b8 f   qt-mt323:qt-mt323.dll
 0001:000016be       ?setPalette@QWidget@@UAEXABVQPalette@@@Z 100026be f   qt-mt323:qt-mt323.dll
 0001:000016c4       ?setPaletteBackgroundColor@QWidget@@UAEXABVQColor@@@Z 100026c4 f   qt-mt323:qt-mt323.dll
 0001:000016ca       ?setPaletteBackgroundPixmap@QWidget@@UAEXABVQPixmap@@@Z 100026ca f   qt-mt323:qt-mt323.dll
 0001:000016d0       ?setProperty@QObject@@UAE_NPBDABVQVariant@@@Z 100026d0 f   qt-mt323:qt-mt323.dll
 0001:000016d6       ?setResolution@QPaintDevice@@UAEXH@Z 100026d6 f   qt-mt323:qt-mt323.dll
 0001:000016dc       ?setSizeIncrement@QWidget@@UAEXHH@Z 100026dc f   qt-mt323:qt-mt323.dll
 0001:000016e2       ?setSizePolicy@QWidget@@UAEXVQSizePolicy@@@Z 100026e2 f   qt-mt323:qt-mt323.dll
 0001:000016e8       ?setUpdatesEnabled@QWidget@@UAEX_N@Z 100026e8 f   qt-mt323:qt-mt323.dll
 0001:000016ee       ?setWFlags@QWidget@@MAEXI@Z 100026ee f   qt-mt323:qt-mt323.dll
 0001:000016f4       ?setWState@QWidget@@MAEXI@Z 100026f4 f   qt-mt323:qt-mt323.dll
 0001:000016fa       ?show@QWidget@@UAEXXZ      100026fa f   qt-mt323:qt-mt323.dll
 0001:00001700       ?showEvent@QWidget@@MAEXPAVQShowEvent@@@Z 10002700 f   qt-mt323:qt-mt323.dll
 0001:00001706       ?showMaximized@QWidget@@UAEXXZ 10002706 f   qt-mt323:qt-mt323.dll
 0001:0000170c       ?showMinimized@QWidget@@UAEXXZ 1000270c f   qt-mt323:qt-mt323.dll
 0001:00001712       ?showNormal@QWidget@@UAEXXZ 10002712 f   qt-mt323:qt-mt323.dll
 0001:00001718       ?sizeHint@QHBox@@UBE?AVQSize@@XZ 10002718 f   qt-mt323:qt-mt323.dll
 0001:0000171e       ?sizePolicy@QWidget@@UBE?AVQSizePolicy@@XZ 1000271e f   qt-mt323:qt-mt323.dll
 0001:00001724       ?styleChange@QFrame@@MAEXAAVQStyle@@@Z 10002724 f   qt-mt323:qt-mt323.dll
 0001:0000172a       ?tabletEvent@QWidget@@MAEXPAVQTabletEvent@@@Z 1000272a f   qt-mt323:qt-mt323.dll
 0001:00001730       ?timerEvent@QObject@@MAEXPAVQTimerEvent@@@Z 10002730 f   qt-mt323:qt-mt323.dll
 0001:00001736       ?unsetCursor@QWidget@@UAEXXZ 10002736 f   qt-mt323:qt-mt323.dll
 0001:0000173c       ?updateMask@QWidget@@MAEXXZ 1000273c f   qt-mt323:qt-mt323.dll
 0001:00001742       ?wheelEvent@QWidget@@MAEXPAVQWheelEvent@@@Z 10002742 f   qt-mt323:qt-mt323.dll
 0001:00001748       ?winEvent@QWidget@@MAE_NPAUtagMSG@@@Z 10002748 f   qt-mt323:qt-mt323.dll
 0001:0000174e       ?windowActivationChange@QWidget@@MAEX_N@Z 1000274e f   qt-mt323:qt-mt323.dll
 0001:00001754       ?addItem@QBoxLayout@@UAEXPAVQLayoutItem@@@Z 10002754 f   qt-mt323:qt-mt323.dll
 0001:0000175a       ?childEvent@QLayout@@MAEXPAVQChildEvent@@@Z 1000275a f   qt-mt323:qt-mt323.dll
 0001:00001760       ?className@QHBoxLayout@@UBEPBDXZ 10002760 f   qt-mt323:qt-mt323.dll
 0001:00001766       ?className@QLabel@@UBEPBDXZ 10002766 f   qt-mt323:qt-mt323.dll
 0001:0000176c       ?className@QPushButton@@UBEPBDXZ 1000276c f   qt-mt323:qt-mt323.dll
 0001:00001772       ?className@QVBoxLayout@@UBEPBDXZ 10002772 f   qt-mt323:qt-mt323.dll
 0001:00001778       ?drawButton@QPushButton@@MAEXPAVQPainter@@@Z 10002778 f   qt-mt323:qt-mt323.dll
 0001:0000177e       ?drawButtonLabel@QPushButton@@MAEXPAVQPainter@@@Z 1000277e f   qt-mt323:qt-mt323.dll
 0001:00001784       ?drawContents@QLabel@@MAEXPAVQPainter@@@Z 10002784 f   qt-mt323:qt-mt323.dll
 0001:0000178a       ?enabledChange@QButton@@MAEX_N@Z 1000278a f   qt-mt323:qt-mt323.dll
 0001:00001790       ?event@QObject@@UAE_NPAVQEvent@@@Z 10002790 f   qt-mt323:qt-mt323.dll
 0001:00001796       ?eventFilter@QLayout@@MAE_NPAVQObject@@PAVQEvent@@@Z 10002796 f   qt-mt323:qt-mt323.dll
 0001:0000179c       ?expanding@QBoxLayout@@UBE?AW4ExpandData@QSizePolicy@@XZ 1000279c f   qt-mt323:qt-mt323.dll
 0001:000017a2       ?expanding@QSpacerItem@@UBE?AW4ExpandData@QSizePolicy@@XZ 100027a2 f   qt-mt323:qt-mt323.dll
 0001:000017a8       ?focusInEvent@QPushButton@@MAEXPAVQFocusEvent@@@Z 100027a8 f   qt-mt323:qt-mt323.dll
 0001:000017ae       ?focusOutEvent@QPushButton@@MAEXPAVQFocusEvent@@@Z 100027ae f   qt-mt323:qt-mt323.dll
 0001:000017b4       ?fontChange@QLabel@@MAEXABVQFont@@@Z 100027b4 f   qt-mt323:qt-mt323.dll
 0001:000017ba       ?frameChanged@QFrame@@MAEXXZ 100027ba f   qt-mt323:qt-mt323.dll
 0001:000017c0       ?geometry@QLayout@@UBE?AVQRect@@XZ 100027c0 f   qt-mt323:qt-mt323.dll
 0001:000017c6       ?geometry@QSpacerItem@@UBE?AVQRect@@XZ 100027c6 f   qt-mt323:qt-mt323.dll
 0001:000017cc       ?hasHeightForWidth@QBoxLayout@@UBE_NXZ 100027cc f   qt-mt323:qt-mt323.dll
 0001:000017d2       ?hasHeightForWidth@QLayoutItem@@UBE_NXZ 100027d2 f   qt-mt323:qt-mt323.dll
 0001:000017d8       ?heightForWidth@QBoxLayout@@UBEHH@Z 100027d8 f   qt-mt323:qt-mt323.dll
 0001:000017de       ?heightForWidth@QLabel@@UBEHH@Z 100027de f   qt-mt323:qt-mt323.dll
 0001:000017e4       ?heightForWidth@QLayoutItem@@UBEHH@Z 100027e4 f   qt-mt323:qt-mt323.dll
 0001:000017ea       ?hitButton@QButton@@MBE_NABVQPoint@@@Z 100027ea f   qt-mt323:qt-mt323.dll
 0001:000017f0       ?invalidate@QBoxLayout@@UAEXXZ 100027f0 f   qt-mt323:qt-mt323.dll
 0001:000017f6       ?invalidate@QLayoutItem@@UAEXXZ 100027f6 f   qt-mt323:qt-mt323.dll
 0001:000017fc       ?isEmpty@QLayout@@UBE_NXZ  100027fc f   qt-mt323:qt-mt323.dll
 0001:00001802       ?isEmpty@QSpacerItem@@UBE_NXZ 10002802 f   qt-mt323:qt-mt323.dll
 0001:00001808       ?iterator@QBoxLayout@@UAE?AVQLayoutIterator@@XZ 10002808 f   qt-mt323:qt-mt323.dll
 0001:0000180e       ?iterator@QLayoutItem@@UAE?AVQLayoutIterator@@XZ 1000280e f   qt-mt323:qt-mt323.dll
 0001:00001814       ?keyPressEvent@QButton@@MAEXPAVQKeyEvent@@@Z 10002814 f   qt-mt323:qt-mt323.dll
 0001:0000181a       ?keyReleaseEvent@QButton@@MAEXPAVQKeyEvent@@@Z 1000281a f   qt-mt323:qt-mt323.dll
 0001:00001820       ?layout@QLayout@@UAEPAV1@XZ 10002820 f   qt-mt323:qt-mt323.dll
 0001:00001826       ?layout@QLayoutItem@@UAEPAVQLayout@@XZ 10002826 f   qt-mt323:qt-mt323.dll
 0001:0000182c       ?maximumSize@QBoxLayout@@UBE?AVQSize@@XZ 1000282c f   qt-mt323:qt-mt323.dll
 0001:00001832       ?maximumSize@QSpacerItem@@UBE?AVQSize@@XZ 10002832 f   qt-mt323:qt-mt323.dll
 0001:00001838       ?metaObject@QHBoxLayout@@UBEPAVQMetaObject@@XZ 10002838 f   qt-mt323:qt-mt323.dll
 0001:0000183e       ?metaObject@QLabel@@UBEPAVQMetaObject@@XZ 1000283e f   qt-mt323:qt-mt323.dll
 0001:00001844       ?metaObject@QPushButton@@UBEPAVQMetaObject@@XZ 10002844 f   qt-mt323:qt-mt323.dll
 0001:0000184a       ?metaObject@QVBoxLayout@@UBEPAVQMetaObject@@XZ 1000284a f   qt-mt323:qt-mt323.dll
 0001:00001850       ?minimumSize@QBoxLayout@@UBE?AVQSize@@XZ 10002850 f   qt-mt323:qt-mt323.dll
 0001:00001856       ?minimumSize@QSpacerItem@@UBE?AVQSize@@XZ 10002856 f   qt-mt323:qt-mt323.dll
 0001:0000185c       ?minimumSizeHint@QLabel@@UBE?AVQSize@@XZ 1000285c f   qt-mt323:qt-mt323.dll
 0001:00001862       ?mouseMoveEvent@QButton@@MAEXPAVQMouseEvent@@@Z 10002862 f   qt-mt323:qt-mt323.dll
 0001:00001868       ?mousePressEvent@QButton@@MAEXPAVQMouseEvent@@@Z 10002868 f   qt-mt323:qt-mt323.dll
 0001:0000186e       ?mouseReleaseEvent@QButton@@MAEXPAVQMouseEvent@@@Z 1000286e f   qt-mt323:qt-mt323.dll
 0001:00001874       ?move@QPushButton@@UAEXHH@Z 10002874 f   qt-mt323:qt-mt323.dll
 0001:0000187a       ?paintEvent@QButton@@MAEXPAVQPaintEvent@@@Z 1000287a f   qt-mt323:qt-mt323.dll
 0001:00001880       ?paintEvent@QWidget@@MAEXPAVQPaintEvent@@@Z 10002880 f   qt-mt323:qt-mt323.dll
 0001:00001886       ?qt_cast@QHBoxLayout@@UAEPAXPBD@Z 10002886 f   qt-mt323:qt-mt323.dll
 0001:0000188c       ?qt_cast@QLabel@@UAEPAXPBD@Z 1000288c f   qt-mt323:qt-mt323.dll
 0001:00001892       ?qt_cast@QPushButton@@UAEPAXPBD@Z 10002892 f   qt-mt323:qt-mt323.dll
 0001:00001898       ?qt_cast@QVBoxLayout@@UAEPAXPBD@Z 10002898 f   qt-mt323:qt-mt323.dll
 0001:0000189e       ?qt_emit@QHBoxLayout@@UAE_NHPAUQUObject@@@Z 1000289e f   qt-mt323:qt-mt323.dll
 0001:000018a4       ?qt_emit@QLabel@@UAE_NHPAUQUObject@@@Z 100028a4 f   qt-mt323:qt-mt323.dll
 0001:000018aa       ?qt_emit@QPushButton@@UAE_NHPAUQUObject@@@Z 100028aa f   qt-mt323:qt-mt323.dll
 0001:000018b0       ?qt_emit@QVBoxLayout@@UAE_NHPAUQUObject@@@Z 100028b0 f   qt-mt323:qt-mt323.dll
 0001:000018b6       ?qt_invoke@QHBoxLayout@@UAE_NHPAUQUObject@@@Z 100028b6 f   qt-mt323:qt-mt323.dll
 0001:000018bc       ?qt_invoke@QLabel@@UAE_NHPAUQUObject@@@Z 100028bc f   qt-mt323:qt-mt323.dll
 0001:000018c2       ?qt_invoke@QPushButton@@UAE_NHPAUQUObject@@@Z 100028c2 f   qt-mt323:qt-mt323.dll
 0001:000018c8       ?qt_invoke@QVBoxLayout@@UAE_NHPAUQUObject@@@Z 100028c8 f   qt-mt323:qt-mt323.dll
 0001:000018ce       ?qt_property@QHBoxLayout@@UAE_NHHPAVQVariant@@@Z 100028ce f   qt-mt323:qt-mt323.dll
 0001:000018d4       ?qt_property@QLabel@@UAE_NHHPAVQVariant@@@Z 100028d4 f   qt-mt323:qt-mt323.dll
 0001:000018da       ?qt_property@QPushButton@@UAE_NHHPAVQVariant@@@Z 100028da f   qt-mt323:qt-mt323.dll
 0001:000018e0       ?qt_property@QVBoxLayout@@UAE_NHHPAVQVariant@@@Z 100028e0 f   qt-mt323:qt-mt323.dll
 0001:000018e6       ?resize@QPushButton@@UAEXHH@Z 100028e6 f   qt-mt323:qt-mt323.dll
 0001:000018ec       ?resizeEvent@QLabel@@MAEXPAVQResizeEvent@@@Z 100028ec f   qt-mt323:qt-mt323.dll
 0001:000018f2       ?resizeEvent@QPushButton@@MAEXPAVQResizeEvent@@@Z 100028f2 f   qt-mt323:qt-mt323.dll
 0001:000018f8       ?resizeEvent@QWidget@@MAEXPAVQResizeEvent@@@Z 100028f8 f   qt-mt323:qt-mt323.dll
 0001:000018fe       ?setAccel@QButton@@UAEXABVQKeySequence@@@Z 100028fe f   qt-mt323:qt-mt323.dll
 0001:00001904       ?setAlignment@QLabel@@UAEXH@Z 10002904 f   qt-mt323:qt-mt323.dll
 0001:0000190a       ?setAlignment@QLayoutItem@@UAEXH@Z 1000290a f   qt-mt323:qt-mt323.dll
 0001:00001910       ?setAutoAdd@QLayout@@UAEX_N@Z 10002910 f   qt-mt323:qt-mt323.dll
 0001:00001916       ?setAutoDefault@QPushButton@@UAEX_N@Z 10002916 f   qt-mt323:qt-mt323.dll
 0001:0000191c       ?setAutoRepeat@QButton@@UAEX_N@Z 1000291c f   qt-mt323:qt-mt323.dll
 0001:00001922       ?setAutoResize@QLabel@@UAEX_N@Z 10002922 f   qt-mt323:qt-mt323.dll
 0001:00001928       ?setBuddy@QLabel@@UAEXPAVQWidget@@@Z 10002928 f   qt-mt323:qt-mt323.dll
 0001:0000192e       ?setDefault@QPushButton@@UAEX_N@Z 1000292e f   qt-mt323:qt-mt323.dll
 0001:00001934       ?setDown@QButton@@UAEX_N@Z 10002934 f   qt-mt323:qt-mt323.dll
 0001:0000193a       ?setFont@QLabel@@UAEXABVQFont@@@Z 1000293a f   qt-mt323:qt-mt323.dll
 0001:00001940       ?setGeometry@QBoxLayout@@UAEXABVQRect@@@Z 10002940 f   qt-mt323:qt-mt323.dll
 0001:00001946       ?setGeometry@QPushButton@@UAEXABVQRect@@@Z 10002946 f   qt-mt323:qt-mt323.dll
 0001:0000194c       ?setGeometry@QPushButton@@UAEXHHHH@Z 1000294c f   qt-mt323:qt-mt323.dll
 0001:00001952       ?setGeometry@QSpacerItem@@UAEXABVQRect@@@Z 10002952 f   qt-mt323:qt-mt323.dll
 0001:00001958       ?setGroup@QButton@@EAEXPAVQButtonGroup@@@Z 10002958 f   qt-mt323:qt-mt323.dll
 0001:0000195e       ?setIsMenuButton@QPushButton@@UAEX_N@Z 1000295e f   qt-mt323:qt-mt323.dll
 0001:00001964       ?setMargin@QLayout@@UAEXH@Z 10002964 f   qt-mt323:qt-mt323.dll
 0001:0000196a       ?setMenuBar@QLayout@@UAEXPAVQMenuBar@@@Z 1000296a f   qt-mt323:qt-mt323.dll
 0001:00001970       ?setMovie@QLabel@@UAEXABVQMovie@@@Z 10002970 f   qt-mt323:qt-mt323.dll
 0001:00001976       ?setName@QObject@@UAEXPBD@Z 10002976 f   qt-mt323:qt-mt323.dll
 0001:0000197c       ?setNum@QLabel@@UAEXH@Z    1000297c f   qt-mt323:qt-mt323.dll
 0001:00001982       ?setNum@QLabel@@UAEXN@Z    10002982 f   qt-mt323:qt-mt323.dll
 0001:00001988       ?setOn@QPushButton@@UAEX_N@Z 10002988 f   qt-mt323:qt-mt323.dll
 0001:0000198e       ?setPicture@QLabel@@UAEXABVQPicture@@@Z 1000298e f   qt-mt323:qt-mt323.dll
 0001:00001994       ?setPixmap@QButton@@UAEXABVQPixmap@@@Z 10002994 f   qt-mt323:qt-mt323.dll
 0001:0000199a       ?setPixmap@QLabel@@UAEXABVQPixmap@@@Z 1000299a f   qt-mt323:qt-mt323.dll
 0001:000019a0       ?setSpacing@QLayout@@UAEXH@Z 100029a0 f   qt-mt323:qt-mt323.dll
 0001:000019a6       ?setState@QButton@@MAEXW4ToggleState@1@@Z 100029a6 f   qt-mt323:qt-mt323.dll
 0001:000019ac       ?setText@QButton@@UAEXABVQString@@@Z 100029ac f   qt-mt323:qt-mt323.dll
 0001:000019b2       ?setText@QLabel@@UAEXABVQString@@@Z 100029b2 f   qt-mt323:qt-mt323.dll
 0001:000019b8       ?setToggleType@QButton@@MAEXW4ToggleType@1@@Z 100029b8 f   qt-mt323:qt-mt323.dll
 0001:000019be       ?sizeHint@QBoxLayout@@UBE?AVQSize@@XZ 100029be f   qt-mt323:qt-mt323.dll
 0001:000019c4       ?sizeHint@QLabel@@UBE?AVQSize@@XZ 100029c4 f   qt-mt323:qt-mt323.dll
 0001:000019ca       ?sizeHint@QPushButton@@UBE?AVQSize@@XZ 100029ca f   qt-mt323:qt-mt323.dll
 0001:000019d0       ?sizeHint@QSpacerItem@@UBE?AVQSize@@XZ 100029d0 f   qt-mt323:qt-mt323.dll
 0001:000019d6       ?sizeHint@QWidget@@UBE?AVQSize@@XZ 100029d6 f   qt-mt323:qt-mt323.dll
 0001:000019dc       ?spacerItem@QLayoutItem@@UAEPAVQSpacerItem@@XZ 100029dc f   qt-mt323:qt-mt323.dll
 0001:000019e2       ?spacerItem@QSpacerItem@@UAEPAV1@XZ 100029e2 f   qt-mt323:qt-mt323.dll
 0001:000019e8       ?styleChange@QWidget@@MAEXAAVQStyle@@@Z 100029e8 f   qt-mt323:qt-mt323.dll
 0001:000019ee       ?updateMask@QPushButton@@MAEXXZ 100029ee f   qt-mt323:qt-mt323.dll
 0001:000019f4       ?widget@QLayoutItem@@UAEPAVQWidget@@XZ 100029f4 f   qt-mt323:qt-mt323.dll
 0001:000019fa       ??_M@YGXPAXIHP6EX0@Z@Z     100029fa f   MSVCRT:ehvecdtr.obj
 0001:00001a69       ?__ArrayUnwind@@YGXPAXIHP6EX0@Z@Z 10002a69 f   MSVCRT:ehvecdtr.obj
 0001:00001ac8       ??2@YAPAXI@Z               10002ac8 f   MSVCRT:MSVCR120.dll
 0001:00001ace       ??3@YAXPAX@Z               10002ace f   MSVCRT:MSVCR120.dll
 0001:00001ad4       ___atonexitinit            10002ad4 f   MSVCRT:atonexit.obj
 0001:00001b10       __onexit                   10002b10 f   MSVCRT:atonexit.obj
 0001:00001bb9       _atexit                    10002bb9 f   MSVCRT:atonexit.obj
 0001:00001bce       @__security_check_cookie@4 10002bce f   MSVCRT:secchk.obj
 0001:00001bde       ___CxxFrameHandler3        10002bde f   MSVCRT:MSVCR120.dll
 0001:00001be4       ??_Etype_info@@UAEPAXI@Z   10002be4 f i MSVCRT:ti_inst.obj
 0001:00001c7a       __CRT_INIT@12              10002c7a f   MSVCRT:crtdll.obj
 0001:00001e71       __DllMainCRTStartup@12     10002e71 f   MSVCRT:crtdll.obj
 0001:00001fc8       ?terminate@@YAXXZ          10002fc8 f   MSVCRT:MSVCR120.dll
 0001:00001fd0       __SEH_prolog4              10002fd0 f   MSVCRT:sehprolg4.obj
 0001:00002015       __SEH_epilog4              10003015 f   MSVCRT:sehprolg4.obj
 0001:00002029       __except_handler4          10003029 f   MSVCRT:chandler4gs.obj
 0001:0000204c       __lock                     1000304c f   MSVCRT:MSVCR120.dll
 0001:00002052       __unlock                   10003052 f   MSVCRT:MSVCR120.dll
 0001:00002058       ___dllonexit               10003058 f   MSVCRT:MSVCR120.dll
 0001:0000205e       ___raise_securityfailure   1000305e f   MSVCRT:gs_report.obj
 0001:0000209b       ___report_gsfailure        1000309b f   MSVCRT:gs_report.obj
 0001:00002196       ??1type_info@@UAE@XZ       10003196 f   MSVCRT:MSVCR120.dll
 0001:0000219c       ___CppXcptFilter           1000319c f   MSVCRT:MSVCR120.dll
 0001:000021a2       __amsg_exit                100031a2 f   MSVCRT:MSVCR120.dll
 0001:000021b0       __FindPESection            100031b0 f   MSVCRT:pesect.obj
 0001:00002200       __IsNonwritableInCurrentImage 10003200 f   MSVCRT:pesect.obj
 0001:000022c0       __ValidateImageBase        100032c0 f   MSVCRT:pesect.obj
 0001:000022f1       ___security_init_cookie    100032f1 f   MSVCRT:gs_support.obj
 0001:0000238d       __RTC_Initialize           1000338d f   MSVCRT:initsect.obj
 0001:000023ad       __RTC_Terminate            100033ad f   MSVCRT:initsect.obj
 0001:000023ce       __initterm                 100033ce f   MSVCRT:MSVCR120.dll
 0001:000023d4       __initterm_e               100033d4 f   MSVCRT:MSVCR120.dll
 0001:000023da       ___clean_type_info_names   100033da f   MSVCRT:tncleanup.obj
 0001:000023e6       __except_handler4_common   100033e6 f   MSVCRT:MSVCR120.dll
 0001:000023ec       __crt_debugger_hook        100033ec f   MSVCRT:MSVCR120.dll
 0001:000023f2       ___crtUnhandledException   100033f2 f   MSVCRT:MSVCR120.dll
 0001:000023f8       ___crtTerminateProcess     100033f8 f   MSVCRT:MSVCR120.dll
 0001:000023fe       ___clean_type_info_names_internal 100033fe f   MSVCRT:MSVCR120.dll
 0001:00002404       _IsProcessorFeaturePresent@4 10003404 f   kernel32:KERNEL32.dll
 0002:00000000       __imp__GetCurrentThreadId@0 10004000     kernel32:KERNEL32.dll
 0002:00000004       __imp__GetCurrentProcessId@0 10004004     kernel32:KERNEL32.dll
 0002:00000008       __imp__QueryPerformanceCounter@4 10004008     kernel32:KERNEL32.dll
 0002:0000000c       __imp__IsProcessorFeaturePresent@4 1000400c     kernel32:KERNEL32.dll
 0002:00000010       __imp__IsDebuggerPresent@0 10004010     kernel32:KERNEL32.dll
 0002:00000014       __imp__DecodePointer@4     10004014     kernel32:KERNEL32.dll
 0002:00000018       __imp__EncodePointer@4     10004018     kernel32:KERNEL32.dll
 0002:0000001c       __imp__GetSystemTimeAsFileTime@4 1000401c     kernel32:KERNEL32.dll
 0002:00000020       \177KERNEL32_NULL_THUNK_DATA 10004020     kernel32:KERNEL32.dll
 0002:00000024       __imp____clean_type_info_names_internal 10004024     MSVCRT:MSVCR120.dll
 0002:00000028       __imp____crtUnhandledException 10004028     MSVCRT:MSVCR120.dll
 0002:0000002c       __imp___crt_debugger_hook  1000402c     MSVCRT:MSVCR120.dll
 0002:00000030       __imp___except_handler4_common 10004030     MSVCRT:MSVCR120.dll
 0002:00000034       __imp___initterm_e         10004034     MSVCRT:MSVCR120.dll
 0002:00000038       __imp___initterm           10004038     MSVCRT:MSVCR120.dll
 0002:0000003c       __imp___malloc_crt         1000403c     MSVCRT:MSVCR120.dll
 0002:00000040       __imp__free                10004040     MSVCRT:MSVCR120.dll
 0002:00000044       __imp___amsg_exit          10004044     MSVCRT:MSVCR120.dll
 0002:00000048       __imp____CppXcptFilter     10004048     MSVCRT:MSVCR120.dll
 0002:0000004c       __imp_??1type_info@@UAE@XZ 1000404c     MSVCRT:MSVCR120.dll
 0002:00000050       __imp___onexit             10004050     MSVCRT:MSVCR120.dll
 0002:00000054       __imp____dllonexit         10004054     MSVCRT:MSVCR120.dll
 0002:00000058       __imp___calloc_crt         10004058     MSVCRT:MSVCR120.dll
 0002:0000005c       __imp___unlock             1000405c     MSVCRT:MSVCR120.dll
 0002:00000060       __imp___lock               10004060     MSVCRT:MSVCR120.dll
 0002:00000064       __imp_?terminate@@YAXXZ    10004064     MSVCRT:MSVCR120.dll
 0002:00000068       __imp____CxxFrameHandler3  10004068     MSVCRT:MSVCR120.dll
 0002:0000006c       __imp_??3@YAXPAX@Z         1000406c     MSVCRT:MSVCR120.dll
 0002:00000070       __imp_??2@YAPAXI@Z         10004070     MSVCRT:MSVCR120.dll
 0002:00000074       __imp____crtTerminateProcess 10004074     MSVCRT:MSVCR120.dll
 0002:00000078       \177MSVCR120_NULL_THUNK_DATA 10004078     MSVCRT:MSVCR120.dll
 0002:0000007c       __imp_??1QStringList@@QAE@XZ 1000407c     qt-mt323:qt-mt323.dll
 0002:00000080       __imp_??4QStringList@@QAEAAV0@ABV0@@Z 10004080     qt-mt323:qt-mt323.dll
 0002:00000084       __imp_??1QWidget@@UAE@XZ   10004084     qt-mt323:qt-mt323.dll
 0002:00000088       __imp_??4QFrame@@QAEAAV0@ABV0@@Z 10004088     qt-mt323:qt-mt323.dll
 0002:0000008c       __imp_?getItem@QInputDialog@@SA?AVQString@@ABV2@0ABVQStringList@@H_NPA_NPAVQWidget@@PBD@Z 1000408c     qt-mt323:qt-mt323.dll
 0002:00000090       __imp_??0QVBox@@QAE@PAVQWidget@@PBDI@Z 10004090     qt-mt323:qt-mt323.dll
 0002:00000094       __imp_??1QVBox@@UAE@XZ     10004094     qt-mt323:qt-mt323.dll
 0002:00000098       __imp_?adjustSize@QWidget@@UAEXXZ 10004098     qt-mt323:qt-mt323.dll
 0002:0000009c       __imp_?checkConnectArgs@QObject@@MAE_NPBDPBV1@0@Z 1000409c     qt-mt323:qt-mt323.dll
 0002:000000a0       __imp_?childEvent@QObject@@MAEXPAVQChildEvent@@@Z 100040a0     qt-mt323:qt-mt323.dll
 0002:000000a4       __imp_?close@QWidget@@UAE_N_N@Z 100040a4     qt-mt323:qt-mt323.dll
 0002:000000a8       __imp_?closeEvent@QWidget@@MAEXPAVQCloseEvent@@@Z 100040a8     qt-mt323:qt-mt323.dll
 0002:000000ac       __imp_?cmd@QPaintDevice@@MAE_NHPAVQPainter@@PATQPDevCmdParam@@@Z 100040ac     qt-mt323:qt-mt323.dll
 0002:000000b0       __imp_?connectNotify@QObject@@MAEXPBD@Z 100040b0     qt-mt323:qt-mt323.dll
 0002:000000b4       __imp_?contextMenuEvent@QWidget@@MAEXPAVQContextMenuEvent@@@Z 100040b4     qt-mt323:qt-mt323.dll
 0002:000000b8       __imp_?create@QWidget@@MAEXPAUHWND__@@_N1@Z 100040b8     qt-mt323:qt-mt323.dll
 0002:000000bc       __imp_?customEvent@QObject@@MAEXPAVQCustomEvent@@@Z 100040bc     qt-mt323:qt-mt323.dll
 0002:000000c0       __imp_?customWhatsThis@QWidget@@UBE_NXZ 100040c0     qt-mt323:qt-mt323.dll
 0002:000000c4       __imp_?destroy@QWidget@@MAEX_N0@Z 100040c4     qt-mt323:qt-mt323.dll
 0002:000000c8       __imp_?disconnectNotify@QObject@@MAEXPBD@Z 100040c8     qt-mt323:qt-mt323.dll
 0002:000000cc       __imp_?dragEnterEvent@QWidget@@MAEXPAVQDragEnterEvent@@@Z 100040cc     qt-mt323:qt-mt323.dll
 0002:000000d0       __imp_?dragLeaveEvent@QWidget@@MAEXPAVQDragLeaveEvent@@@Z 100040d0     qt-mt323:qt-mt323.dll
 0002:000000d4       __imp_?dragMoveEvent@QWidget@@MAEXPAVQDragMoveEvent@@@Z 100040d4     qt-mt323:qt-mt323.dll
 0002:000000d8       __imp_?drawContents@QFrame@@MAEXPAVQPainter@@@Z 100040d8     qt-mt323:qt-mt323.dll
 0002:000000dc       __imp_?drawFrame@QFrame@@MAEXPAVQPainter@@@Z 100040dc     qt-mt323:qt-mt323.dll
 0002:000000e0       __imp_?dropEvent@QWidget@@MAEXPAVQDropEvent@@@Z 100040e0     qt-mt323:qt-mt323.dll
 0002:000000e4       __imp_?enabledChange@QWidget@@MAEX_N@Z 100040e4     qt-mt323:qt-mt323.dll
 0002:000000e8       __imp_?enterEvent@QWidget@@MAEXPAVQEvent@@@Z 100040e8     qt-mt323:qt-mt323.dll
 0002:000000ec       __imp_?event@QWidget@@MAE_NPAVQEvent@@@Z 100040ec     qt-mt323:qt-mt323.dll
 0002:000000f0       __imp_?eventFilter@QObject@@UAE_NPAV1@PAVQEvent@@@Z 100040f0     qt-mt323:qt-mt323.dll
 0002:000000f4       __imp_?focusInEvent@QWidget@@MAEXPAVQFocusEvent@@@Z 100040f4     qt-mt323:qt-mt323.dll
 0002:000000f8       __imp_?focusNextPrevChild@QWidget@@MAE_N_N@Z 100040f8     qt-mt323:qt-mt323.dll
 0002:000000fc       __imp_?focusOutEvent@QWidget@@MAEXPAVQFocusEvent@@@Z 100040fc     qt-mt323:qt-mt323.dll
 0002:00000100       __imp_?fontChange@QWidget@@MAEXABVQFont@@@Z 10004100     qt-mt323:qt-mt323.dll
 0002:00000104       __imp_?fontInf@QPaintDevice@@MBEHPAVQFont@@H@Z 10004104     qt-mt323:qt-mt323.dll
 0002:00000108       __imp_?fontMet@QPaintDevice@@MBEHPAVQFont@@HPBDH@Z 10004108     qt-mt323:qt-mt323.dll
 0002:0000010c       __imp_?frameChanged@QHBox@@MAEXXZ 1000410c     qt-mt323:qt-mt323.dll
 0002:00000110       __imp_?handle@QPaintDevice@@UBEPAUHDC__@@XZ 10004110     qt-mt323:qt-mt323.dll
 0002:00000114       __imp_?heightForWidth@QWidget@@UBEHH@Z 10004114     qt-mt323:qt-mt323.dll
 0002:00000118       __imp_?hide@QWidget@@UAEXXZ 10004118     qt-mt323:qt-mt323.dll
 0002:0000011c       __imp_?hideEvent@QWidget@@MAEXPAVQHideEvent@@@Z 1000411c     qt-mt323:qt-mt323.dll
 0002:00000120       __imp_?imComposeEvent@QWidget@@MAEXPAVQIMEvent@@@Z 10004120     qt-mt323:qt-mt323.dll
 0002:00000124       __imp_?imEndEvent@QWidget@@MAEXPAVQIMEvent@@@Z 10004124     qt-mt323:qt-mt323.dll
 0002:00000128       __imp_?imStartEvent@QWidget@@MAEXPAVQIMEvent@@@Z 10004128     qt-mt323:qt-mt323.dll
 0002:0000012c       __imp_?insertChild@QObject@@UAEXPAV1@@Z 1000412c     qt-mt323:qt-mt323.dll
 0002:00000130       __imp_?keyPressEvent@QWidget@@MAEXPAVQKeyEvent@@@Z 10004130     qt-mt323:qt-mt323.dll
 0002:00000134       __imp_?keyReleaseEvent@QWidget@@MAEXPAVQKeyEvent@@@Z 10004134     qt-mt323:qt-mt323.dll
 0002:00000138       __imp_?leaveEvent@QWidget@@MAEXPAVQEvent@@@Z 10004138     qt-mt323:qt-mt323.dll
 0002:0000013c       __imp_?metric@QWidget@@MBEHH@Z 1000413c     qt-mt323:qt-mt323.dll
 0002:00000140       __imp_?minimumSizeHint@QWidget@@UBE?AVQSize@@XZ 10004140     qt-mt323:qt-mt323.dll
 0002:00000144       __imp_?mouseDoubleClickEvent@QWidget@@MAEXPAVQMouseEvent@@@Z 10004144     qt-mt323:qt-mt323.dll
 0002:00000148       __imp_?mouseMoveEvent@QWidget@@MAEXPAVQMouseEvent@@@Z 10004148     qt-mt323:qt-mt323.dll
 0002:0000014c       __imp_?mousePressEvent@QWidget@@MAEXPAVQMouseEvent@@@Z 1000414c     qt-mt323:qt-mt323.dll
 0002:00000150       __imp_?mouseReleaseEvent@QWidget@@MAEXPAVQMouseEvent@@@Z 10004150     qt-mt323:qt-mt323.dll
 0002:00000154       __imp_?move@QWidget@@UAEXHH@Z 10004154     qt-mt323:qt-mt323.dll
 0002:00000158       __imp_?moveEvent@QWidget@@MAEXPAVQMoveEvent@@@Z 10004158     qt-mt323:qt-mt323.dll
 0002:0000015c       __imp_?paintEvent@QFrame@@MAEXPAVQPaintEvent@@@Z 1000415c     qt-mt323:qt-mt323.dll
 0002:00000160       __imp_?paletteChange@QWidget@@MAEXABVQPalette@@@Z 10004160     qt-mt323:qt-mt323.dll
 0002:00000164       __imp_?polish@QWidget@@UAEXXZ 10004164     qt-mt323:qt-mt323.dll
 0002:00000168       __imp_?property@QObject@@UBE?AVQVariant@@PBD@Z 10004168     qt-mt323:qt-mt323.dll
 0002:0000016c       __imp_?removeChild@QObject@@UAEXPAV1@@Z 1000416c     qt-mt323:qt-mt323.dll
 0002:00000170       __imp_?reparent@QWidget@@UAEXPAV1@IABVQPoint@@_N@Z 10004170     qt-mt323:qt-mt323.dll
 0002:00000174       __imp_?resize@QWidget@@UAEXHH@Z 10004174     qt-mt323:qt-mt323.dll
 0002:00000178       __imp_?resizeEvent@QFrame@@MAEXPAVQResizeEvent@@@Z 10004178     qt-mt323:qt-mt323.dll
 0002:0000017c       __imp_?resolution@QPaintDevice@@UBEHXZ 1000417c     qt-mt323:qt-mt323.dll
 0002:00000180       __imp_?setAcceptDrops@QWidget@@UAEX_N@Z 10004180     qt-mt323:qt-mt323.dll
 0002:00000184       __imp_?setActiveWindow@QWidget@@UAEXXZ 10004184     qt-mt323:qt-mt323.dll
 0002:00000188       __imp_?setAutoMask@QWidget@@UAEX_N@Z 10004188     qt-mt323:qt-mt323.dll
 0002:0000018c       __imp_?setBackgroundColor@QWidget@@UAEXABVQColor@@@Z 1000418c     qt-mt323:qt-mt323.dll
 0002:00000190       __imp_?setBackgroundMode@QWidget@@UAEXW4BackgroundMode@Qt@@@Z 10004190     qt-mt323:qt-mt323.dll
 0002:00000194       __imp_?setBackgroundOrigin@QWidget@@UAEXW4BackgroundOrigin@1@@Z 10004194     qt-mt323:qt-mt323.dll
 0002:00000198       __imp_?setBackgroundPixmap@QWidget@@UAEXABVQPixmap@@@Z 10004198     qt-mt323:qt-mt323.dll
 0002:0000019c       __imp_?setCaption@QWidget@@UAEXABVQString@@@Z 1000419c     qt-mt323:qt-mt323.dll
 0002:000001a0       __imp_?setCursor@QWidget@@UAEXABVQCursor@@@Z 100041a0     qt-mt323:qt-mt323.dll
 0002:000001a4       __imp_?setEnabled@QWidget@@UAEX_N@Z 100041a4     qt-mt323:qt-mt323.dll
 0002:000001a8       __imp_?setEraseColor@QWidget@@UAEXABVQColor@@@Z 100041a8     qt-mt323:qt-mt323.dll
 0002:000001ac       __imp_?setErasePixmap@QWidget@@UAEXABVQPixmap@@@Z 100041ac     qt-mt323:qt-mt323.dll
 0002:000001b0       __imp_?setFocus@QWidget@@UAEXXZ 100041b0     qt-mt323:qt-mt323.dll
 0002:000001b4       __imp_?setFocusPolicy@QWidget@@UAEXW4FocusPolicy@1@@Z 100041b4     qt-mt323:qt-mt323.dll
 0002:000001b8       __imp_?setFocusProxy@QWidget@@UAEXPAV1@@Z 100041b8     qt-mt323:qt-mt323.dll
 0002:000001bc       __imp_?setFont@QWidget@@UAEXABVQFont@@@Z 100041bc     qt-mt323:qt-mt323.dll
 0002:000001c0       __imp_?setFrameRect@QFrame@@UAEXABVQRect@@@Z 100041c0     qt-mt323:qt-mt323.dll
 0002:000001c4       __imp_?setFrameStyle@QFrame@@UAEXH@Z 100041c4     qt-mt323:qt-mt323.dll
 0002:000001c8       __imp_?setGeometry@QWidget@@UAEXABVQRect@@@Z 100041c8     qt-mt323:qt-mt323.dll
 0002:000001cc       __imp_?setGeometry@QWidget@@UAEXHHHH@Z 100041cc     qt-mt323:qt-mt323.dll
 0002:000001d0       __imp_?setIcon@QWidget@@UAEXABVQPixmap@@@Z 100041d0     qt-mt323:qt-mt323.dll
 0002:000001d4       __imp_?setIconText@QWidget@@UAEXABVQString@@@Z 100041d4     qt-mt323:qt-mt323.dll
 0002:000001d8       __imp_?setKeyCompression@QWidget@@MAEX_N@Z 100041d8     qt-mt323:qt-mt323.dll
 0002:000001dc       __imp_?setLineWidth@QFrame@@UAEXH@Z 100041dc     qt-mt323:qt-mt323.dll
 0002:000001e0       __imp_?setMargin@QFrame@@UAEXH@Z 100041e0     qt-mt323:qt-mt323.dll
 0002:000001e4       __imp_?setMask@QWidget@@UAEXABVQBitmap@@@Z 100041e4     qt-mt323:qt-mt323.dll
 0002:000001e8       __imp_?setMask@QWidget@@UAEXABVQRegion@@@Z 100041e8     qt-mt323:qt-mt323.dll
 0002:000001ec       __imp_?setMaximumSize@QWidget@@UAEXHH@Z 100041ec     qt-mt323:qt-mt323.dll
 0002:000001f0       __imp_?setMicroFocusHint@QWidget@@MAEXHHHH_NPAVQFont@@@Z 100041f0     qt-mt323:qt-mt323.dll
 0002:000001f4       __imp_?setMidLineWidth@QFrame@@UAEXH@Z 100041f4     qt-mt323:qt-mt323.dll
 0002:000001f8       __imp_?setMinimumSize@QWidget@@UAEXHH@Z 100041f8     qt-mt323:qt-mt323.dll
 0002:000001fc       __imp_?setMouseTracking@QWidget@@UAEX_N@Z 100041fc     qt-mt323:qt-mt323.dll
 0002:00000200       __imp_?setName@QWidget@@UAEXPBD@Z 10004200     qt-mt323:qt-mt323.dll
 0002:00000204       __imp_?setPalette@QWidget@@UAEXABVQPalette@@@Z 10004204     qt-mt323:qt-mt323.dll
 0002:00000208       __imp_?setPaletteBackgroundColor@QWidget@@UAEXABVQColor@@@Z 10004208     qt-mt323:qt-mt323.dll
 0002:0000020c       __imp_?setPaletteBackgroundPixmap@QWidget@@UAEXABVQPixmap@@@Z 1000420c     qt-mt323:qt-mt323.dll
 0002:00000210       __imp_?setProperty@QObject@@UAE_NPBDABVQVariant@@@Z 10004210     qt-mt323:qt-mt323.dll
 0002:00000214       __imp_?setResolution@QPaintDevice@@UAEXH@Z 10004214     qt-mt323:qt-mt323.dll
 0002:00000218       __imp_?setSizeIncrement@QWidget@@UAEXHH@Z 10004218     qt-mt323:qt-mt323.dll
 0002:0000021c       __imp_?setSizePolicy@QWidget@@UAEXVQSizePolicy@@@Z 1000421c     qt-mt323:qt-mt323.dll
 0002:00000220       __imp_?setUpdatesEnabled@QWidget@@UAEX_N@Z 10004220     qt-mt323:qt-mt323.dll
 0002:00000224       __imp_?setWFlags@QWidget@@MAEXI@Z 10004224     qt-mt323:qt-mt323.dll
 0002:00000228       __imp_?setWState@QWidget@@MAEXI@Z 10004228     qt-mt323:qt-mt323.dll
 0002:0000022c       __imp_?show@QWidget@@UAEXXZ 1000422c     qt-mt323:qt-mt323.dll
 0002:00000230       __imp_?showEvent@QWidget@@MAEXPAVQShowEvent@@@Z 10004230     qt-mt323:qt-mt323.dll
 0002:00000234       __imp_?showMaximized@QWidget@@UAEXXZ 10004234     qt-mt323:qt-mt323.dll
 0002:00000238       __imp_?showMinimized@QWidget@@UAEXXZ 10004238     qt-mt323:qt-mt323.dll
 0002:0000023c       __imp_?showNormal@QWidget@@UAEXXZ 1000423c     qt-mt323:qt-mt323.dll
 0002:00000240       __imp_?sizeHint@QHBox@@UBE?AVQSize@@XZ 10004240     qt-mt323:qt-mt323.dll
 0002:00000244       __imp_?sizePolicy@QWidget@@UBE?AVQSizePolicy@@XZ 10004244     qt-mt323:qt-mt323.dll
 0002:00000248       __imp_?styleChange@QFrame@@MAEXAAVQStyle@@@Z 10004248     qt-mt323:qt-mt323.dll
 0002:0000024c       __imp_?tabletEvent@QWidget@@MAEXPAVQTabletEvent@@@Z 1000424c     qt-mt323:qt-mt323.dll
 0002:00000250       __imp_?timerEvent@QObject@@MAEXPAVQTimerEvent@@@Z 10004250     qt-mt323:qt-mt323.dll
 0002:00000254       __imp_?unsetCursor@QWidget@@UAEXXZ 10004254     qt-mt323:qt-mt323.dll
 0002:00000258       __imp_?updateMask@QWidget@@MAEXXZ 10004258     qt-mt323:qt-mt323.dll
 0002:0000025c       __imp_?wheelEvent@QWidget@@MAEXPAVQWheelEvent@@@Z 1000425c     qt-mt323:qt-mt323.dll
 0002:00000260       __imp_?winEvent@QWidget@@MAE_NPAUtagMSG@@@Z 10004260     qt-mt323:qt-mt323.dll
 0002:00000264       __imp_?windowActivationChange@QWidget@@MAEX_N@Z 10004264     qt-mt323:qt-mt323.dll
 0002:00000268       __imp_?null@QString@@2V1@A 10004268     qt-mt323:qt-mt323.dll
 0002:0000026c       __imp_?shared_null@QString@@0PAUQStringData@@A 1000426c     qt-mt323:qt-mt323.dll
 0002:00000270       __imp_?fromLatin1@QString@@SA?AV1@PBDH@Z 10004270     qt-mt323:qt-mt323.dll
 0002:00000274       __imp_?fromUtf8@QString@@SA?AV1@PBDH@Z 10004274     qt-mt323:qt-mt323.dll
 0002:00000278       __imp_?qt_cast@QWidget@@UAEPAXPBD@Z 10004278     qt-mt323:qt-mt323.dll
 0002:0000027c       __imp_?qt_invoke@QWidget@@UAE_NHPAUQUObject@@@Z 1000427c     qt-mt323:qt-mt323.dll
 0002:00000280       __imp_?qt_emit@QWidget@@UAE_NHPAUQUObject@@@Z 10004280     qt-mt323:qt-mt323.dll
 0002:00000284       __imp_?qt_property@QWidget@@UAE_NHHPAVQVariant@@@Z 10004284     qt-mt323:qt-mt323.dll
 0002:00000288       __imp_?staticMetaObject@QWidget@@SAPAVQMetaObject@@XZ 10004288     qt-mt323:qt-mt323.dll
 0002:0000028c       __imp_?new_metaobject@QMetaObject@@SAPAV1@PBDPAV1@QBUQMetaData@@H2HQBVQMetaProperty@@HQBUQMetaEnum@@HQBUQClassInfo@@H@Z 1000428c     qt-mt323:qt-mt323.dll
 0002:00000290       __imp_??0QMetaObjectCleanUp@@QAE@PBDP6APAVQMetaObject@@XZ@Z 10004290     qt-mt323:qt-mt323.dll
 0002:00000294       __imp_??1QMetaObjectCleanUp@@QAE@XZ 10004294     qt-mt323:qt-mt323.dll
 0002:00000298       __imp_?setMetaObject@QMetaObjectCleanUp@@QAEXAAPAVQMetaObject@@@Z 10004298     qt-mt323:qt-mt323.dll
 0002:0000029c       __imp_?translate@QApplication@@QBE?AVQString@@PBD00W4Encoding@1@@Z 1000429c     qt-mt323:qt-mt323.dll
 0002:000002a0       __imp_?sort@QStringList@@QAEXXZ 100042a0     qt-mt323:qt-mt323.dll
 0002:000002a4       __imp_??1QVariant@@QAE@XZ  100042a4     qt-mt323:qt-mt323.dll
 0002:000002a8       __imp_??0QVariant@@QAE@_NH@Z 100042a8     qt-mt323:qt-mt323.dll
 0002:000002ac       __imp_??0QWidget@@QAE@PAV0@PBDI@Z 100042ac     qt-mt323:qt-mt323.dll
 0002:000002b0       __imp_?resize@QWidget@@QAEXABVQSize@@@Z 100042b0     qt-mt323:qt-mt323.dll
 0002:000002b4       __imp_??0QPushButton@@QAE@PAVQWidget@@PBD@Z 100042b4     qt-mt323:qt-mt323.dll
 0002:000002b8       __imp_??1QPushButton@@UAE@XZ 100042b8     qt-mt323:qt-mt323.dll
 0002:000002bc       __imp_?setFrameShape@QFrame@@QAEXW4Shape@1@@Z 100042bc     qt-mt323:qt-mt323.dll
 0002:000002c0       __imp_?setFrameShadow@QFrame@@QAEXW4Shadow@1@@Z 100042c0     qt-mt323:qt-mt323.dll
 0002:000002c4       __imp_??0QLabel@@QAE@PAVQWidget@@PBDI@Z 100042c4     qt-mt323:qt-mt323.dll
 0002:000002c8       __imp_??1QLabel@@UAE@XZ    100042c8     qt-mt323:qt-mt323.dll
 0002:000002cc       __imp_??1QLayoutItem@@UAE@XZ 100042cc     qt-mt323:qt-mt323.dll
 0002:000002d0       __imp_?addWidget@QBoxLayout@@QAEXPAVQWidget@@HH@Z 100042d0     qt-mt323:qt-mt323.dll
 0002:000002d4       __imp_?addLayout@QBoxLayout@@QAEXPAVQLayout@@H@Z 100042d4     qt-mt323:qt-mt323.dll
 0002:000002d8       __imp_??0QHBoxLayout@@QAE@PAVQWidget@@HHPBD@Z 100042d8     qt-mt323:qt-mt323.dll
 0002:000002dc       __imp_??1QHBoxLayout@@UAE@XZ 100042dc     qt-mt323:qt-mt323.dll
 0002:000002e0       __imp_??0QVBoxLayout@@QAE@PAVQWidget@@HHPBD@Z 100042e0     qt-mt323:qt-mt323.dll
 0002:000002e4       __imp_??1QVBoxLayout@@UAE@XZ 100042e4     qt-mt323:qt-mt323.dll
 0002:000002e8       __imp_?addItem@QBoxLayout@@UAEXPAVQLayoutItem@@@Z 100042e8     qt-mt323:qt-mt323.dll
 0002:000002ec       __imp_?childEvent@QLayout@@MAEXPAVQChildEvent@@@Z 100042ec     qt-mt323:qt-mt323.dll
 0002:000002f0       __imp_?className@QHBoxLayout@@UBEPBDXZ 100042f0     qt-mt323:qt-mt323.dll
 0002:000002f4       __imp_?className@QLabel@@UBEPBDXZ 100042f4     qt-mt323:qt-mt323.dll
 0002:000002f8       __imp_?className@QPushButton@@UBEPBDXZ 100042f8     qt-mt323:qt-mt323.dll
 0002:000002fc       __imp_?className@QVBoxLayout@@UBEPBDXZ 100042fc     qt-mt323:qt-mt323.dll
 0002:00000300       __imp_?drawButton@QPushButton@@MAEXPAVQPainter@@@Z 10004300     qt-mt323:qt-mt323.dll
 0002:00000304       __imp_?drawButtonLabel@QPushButton@@MAEXPAVQPainter@@@Z 10004304     qt-mt323:qt-mt323.dll
 0002:00000308       __imp_?drawContents@QLabel@@MAEXPAVQPainter@@@Z 10004308     qt-mt323:qt-mt323.dll
 0002:0000030c       __imp_?enabledChange@QButton@@MAEX_N@Z 1000430c     qt-mt323:qt-mt323.dll
 0002:00000310       __imp_?event@QObject@@UAE_NPAVQEvent@@@Z 10004310     qt-mt323:qt-mt323.dll
 0002:00000314       __imp_?eventFilter@QLayout@@MAE_NPAVQObject@@PAVQEvent@@@Z 10004314     qt-mt323:qt-mt323.dll
 0002:00000318       __imp_?expanding@QBoxLayout@@UBE?AW4ExpandData@QSizePolicy@@XZ 10004318     qt-mt323:qt-mt323.dll
 0002:0000031c       __imp_?expanding@QSpacerItem@@UBE?AW4ExpandData@QSizePolicy@@XZ 1000431c     qt-mt323:qt-mt323.dll
 0002:00000320       __imp_?focusInEvent@QPushButton@@MAEXPAVQFocusEvent@@@Z 10004320     qt-mt323:qt-mt323.dll
 0002:00000324       __imp_?focusOutEvent@QPushButton@@MAEXPAVQFocusEvent@@@Z 10004324     qt-mt323:qt-mt323.dll
 0002:00000328       __imp_?fontChange@QLabel@@MAEXABVQFont@@@Z 10004328     qt-mt323:qt-mt323.dll
 0002:0000032c       __imp_?frameChanged@QFrame@@MAEXXZ 1000432c     qt-mt323:qt-mt323.dll
 0002:00000330       __imp_?geometry@QLayout@@UBE?AVQRect@@XZ 10004330     qt-mt323:qt-mt323.dll
 0002:00000334       __imp_?geometry@QSpacerItem@@UBE?AVQRect@@XZ 10004334     qt-mt323:qt-mt323.dll
 0002:00000338       __imp_?hasHeightForWidth@QBoxLayout@@UBE_NXZ 10004338     qt-mt323:qt-mt323.dll
 0002:0000033c       __imp_?hasHeightForWidth@QLayoutItem@@UBE_NXZ 1000433c     qt-mt323:qt-mt323.dll
 0002:00000340       __imp_?heightForWidth@QBoxLayout@@UBEHH@Z 10004340     qt-mt323:qt-mt323.dll
 0002:00000344       __imp_?heightForWidth@QLabel@@UBEHH@Z 10004344     qt-mt323:qt-mt323.dll
 0002:00000348       __imp_?heightForWidth@QLayoutItem@@UBEHH@Z 10004348     qt-mt323:qt-mt323.dll
 0002:0000034c       __imp_?hitButton@QButton@@MBE_NABVQPoint@@@Z 1000434c     qt-mt323:qt-mt323.dll
 0002:00000350       __imp_?invalidate@QBoxLayout@@UAEXXZ 10004350     qt-mt323:qt-mt323.dll
 0002:00000354       __imp_?invalidate@QLayoutItem@@UAEXXZ 10004354     qt-mt323:qt-mt323.dll
 0002:00000358       __imp_?isEmpty@QLayout@@UBE_NXZ 10004358     qt-mt323:qt-mt323.dll
 0002:0000035c       __imp_?isEmpty@QSpacerItem@@UBE_NXZ 1000435c     qt-mt323:qt-mt323.dll
 0002:00000360       __imp_?iterator@QBoxLayout@@UAE?AVQLayoutIterator@@XZ 10004360     qt-mt323:qt-mt323.dll
 0002:00000364       __imp_?iterator@QLayoutItem@@UAE?AVQLayoutIterator@@XZ 10004364     qt-mt323:qt-mt323.dll
 0002:00000368       __imp_?keyPressEvent@QButton@@MAEXPAVQKeyEvent@@@Z 10004368     qt-mt323:qt-mt323.dll
 0002:0000036c       __imp_?keyReleaseEvent@QButton@@MAEXPAVQKeyEvent@@@Z 1000436c     qt-mt323:qt-mt323.dll
 0002:00000370       __imp_?layout@QLayout@@UAEPAV1@XZ 10004370     qt-mt323:qt-mt323.dll
 0002:00000374       __imp_?layout@QLayoutItem@@UAEPAVQLayout@@XZ 10004374     qt-mt323:qt-mt323.dll
 0002:00000378       __imp_?maximumSize@QBoxLayout@@UBE?AVQSize@@XZ 10004378     qt-mt323:qt-mt323.dll
 0002:0000037c       __imp_?maximumSize@QSpacerItem@@UBE?AVQSize@@XZ 1000437c     qt-mt323:qt-mt323.dll
 0002:00000380       __imp_?metaObject@QHBoxLayout@@UBEPAVQMetaObject@@XZ 10004380     qt-mt323:qt-mt323.dll
 0002:00000384       __imp_?metaObject@QLabel@@UBEPAVQMetaObject@@XZ 10004384     qt-mt323:qt-mt323.dll
 0002:00000388       __imp_?metaObject@QPushButton@@UBEPAVQMetaObject@@XZ 10004388     qt-mt323:qt-mt323.dll
 0002:0000038c       __imp_?metaObject@QVBoxLayout@@UBEPAVQMetaObject@@XZ 1000438c     qt-mt323:qt-mt323.dll
 0002:00000390       __imp_?minimumSize@QBoxLayout@@UBE?AVQSize@@XZ 10004390     qt-mt323:qt-mt323.dll
 0002:00000394       __imp_?minimumSize@QSpacerItem@@UBE?AVQSize@@XZ 10004394     qt-mt323:qt-mt323.dll
 0002:00000398       __imp_?minimumSizeHint@QLabel@@UBE?AVQSize@@XZ 10004398     qt-mt323:qt-mt323.dll
 0002:0000039c       __imp_?mouseMoveEvent@QButton@@MAEXPAVQMouseEvent@@@Z 1000439c     qt-mt323:qt-mt323.dll
 0002:000003a0       __imp_?mousePressEvent@QButton@@MAEXPAVQMouseEvent@@@Z 100043a0     qt-mt323:qt-mt323.dll
 0002:000003a4       __imp_?mouseReleaseEvent@QButton@@MAEXPAVQMouseEvent@@@Z 100043a4     qt-mt323:qt-mt323.dll
 0002:000003a8       __imp_?move@QPushButton@@UAEXHH@Z 100043a8     qt-mt323:qt-mt323.dll
 0002:000003ac       __imp_?paintEvent@QButton@@MAEXPAVQPaintEvent@@@Z 100043ac     qt-mt323:qt-mt323.dll
 0002:000003b0       __imp_?paintEvent@QWidget@@MAEXPAVQPaintEvent@@@Z 100043b0     qt-mt323:qt-mt323.dll
 0002:000003b4       __imp_?qt_cast@QHBoxLayout@@UAEPAXPBD@Z 100043b4     qt-mt323:qt-mt323.dll
 0002:000003b8       __imp_?qt_cast@QLabel@@UAEPAXPBD@Z 100043b8     qt-mt323:qt-mt323.dll
 0002:000003bc       __imp_?qt_cast@QPushButton@@UAEPAXPBD@Z 100043bc     qt-mt323:qt-mt323.dll
 0002:000003c0       __imp_?qt_cast@QVBoxLayout@@UAEPAXPBD@Z 100043c0     qt-mt323:qt-mt323.dll
 0002:000003c4       __imp_?qt_emit@QHBoxLayout@@UAE_NHPAUQUObject@@@Z 100043c4     qt-mt323:qt-mt323.dll
 0002:000003c8       __imp_?qt_emit@QLabel@@UAE_NHPAUQUObject@@@Z 100043c8     qt-mt323:qt-mt323.dll
 0002:000003cc       __imp_?qt_emit@QPushButton@@UAE_NHPAUQUObject@@@Z 100043cc     qt-mt323:qt-mt323.dll
 0002:000003d0       __imp_?qt_emit@QVBoxLayout@@UAE_NHPAUQUObject@@@Z 100043d0     qt-mt323:qt-mt323.dll
 0002:000003d4       __imp_?qt_invoke@QHBoxLayout@@UAE_NHPAUQUObject@@@Z 100043d4     qt-mt323:qt-mt323.dll
 0002:000003d8       __imp_?qt_invoke@QLabel@@UAE_NHPAUQUObject@@@Z 100043d8     qt-mt323:qt-mt323.dll
 0002:000003dc       __imp_?qt_invoke@QPushButton@@UAE_NHPAUQUObject@@@Z 100043dc     qt-mt323:qt-mt323.dll
 0002:000003e0       __imp_?qt_invoke@QVBoxLayout@@UAE_NHPAUQUObject@@@Z 100043e0     qt-mt323:qt-mt323.dll
 0002:000003e4       __imp_?qt_property@QHBoxLayout@@UAE_NHHPAVQVariant@@@Z 100043e4     qt-mt323:qt-mt323.dll
 0002:000003e8       __imp_?qt_property@QLabel@@UAE_NHHPAVQVariant@@@Z 100043e8     qt-mt323:qt-mt323.dll
 0002:000003ec       __imp_?qt_property@QPushButton@@UAE_NHHPAVQVariant@@@Z 100043ec     qt-mt323:qt-mt323.dll
 0002:000003f0       __imp_?qt_property@QVBoxLayout@@UAE_NHHPAVQVariant@@@Z 100043f0     qt-mt323:qt-mt323.dll
 0002:000003f4       __imp_?resize@QPushButton@@UAEXHH@Z 100043f4     qt-mt323:qt-mt323.dll
 0002:000003f8       __imp_?resizeEvent@QLabel@@MAEXPAVQResizeEvent@@@Z 100043f8     qt-mt323:qt-mt323.dll
 0002:000003fc       __imp_?resizeEvent@QPushButton@@MAEXPAVQResizeEvent@@@Z 100043fc     qt-mt323:qt-mt323.dll
 0002:00000400       __imp_?resizeEvent@QWidget@@MAEXPAVQResizeEvent@@@Z 10004400     qt-mt323:qt-mt323.dll
 0002:00000404       __imp_?setAccel@QButton@@UAEXABVQKeySequence@@@Z 10004404     qt-mt323:qt-mt323.dll
 0002:00000408       __imp_?setAlignment@QLabel@@UAEXH@Z 10004408     qt-mt323:qt-mt323.dll
 0002:0000040c       __imp_?setAlignment@QLayoutItem@@UAEXH@Z 1000440c     qt-mt323:qt-mt323.dll
 0002:00000410       __imp_?setAutoAdd@QLayout@@UAEX_N@Z 10004410     qt-mt323:qt-mt323.dll
 0002:00000414       __imp_?setAutoDefault@QPushButton@@UAEX_N@Z 10004414     qt-mt323:qt-mt323.dll
 0002:00000418       __imp_?setAutoRepeat@QButton@@UAEX_N@Z 10004418     qt-mt323:qt-mt323.dll
 0002:0000041c       __imp_?setAutoResize@QLabel@@UAEX_N@Z 1000441c     qt-mt323:qt-mt323.dll
 0002:00000420       __imp_?setBuddy@QLabel@@UAEXPAVQWidget@@@Z 10004420     qt-mt323:qt-mt323.dll
 0002:00000424       __imp_?setDefault@QPushButton@@UAEX_N@Z 10004424     qt-mt323:qt-mt323.dll
 0002:00000428       __imp_?setDown@QButton@@UAEX_N@Z 10004428     qt-mt323:qt-mt323.dll
 0002:0000042c       __imp_?setFont@QLabel@@UAEXABVQFont@@@Z 1000442c     qt-mt323:qt-mt323.dll
 0002:00000430       __imp_?setGeometry@QBoxLayout@@UAEXABVQRect@@@Z 10004430     qt-mt323:qt-mt323.dll
 0002:00000434       __imp_?setGeometry@QPushButton@@UAEXABVQRect@@@Z 10004434     qt-mt323:qt-mt323.dll
 0002:00000438       __imp_?setGeometry@QPushButton@@UAEXHHHH@Z 10004438     qt-mt323:qt-mt323.dll
 0002:0000043c       __imp_?setGeometry@QSpacerItem@@UAEXABVQRect@@@Z 1000443c     qt-mt323:qt-mt323.dll
 0002:00000440       __imp_?setGroup@QButton@@EAEXPAVQButtonGroup@@@Z 10004440     qt-mt323:qt-mt323.dll
 0002:00000444       __imp_?setIsMenuButton@QPushButton@@UAEX_N@Z 10004444     qt-mt323:qt-mt323.dll
 0002:00000448       __imp_?setMargin@QLayout@@UAEXH@Z 10004448     qt-mt323:qt-mt323.dll
 0002:0000044c       __imp_?setMenuBar@QLayout@@UAEXPAVQMenuBar@@@Z 1000444c     qt-mt323:qt-mt323.dll
 0002:00000450       __imp_?setMovie@QLabel@@UAEXABVQMovie@@@Z 10004450     qt-mt323:qt-mt323.dll
 0002:00000454       __imp_?setName@QObject@@UAEXPBD@Z 10004454     qt-mt323:qt-mt323.dll
 0002:00000458       __imp_?setNum@QLabel@@UAEXH@Z 10004458     qt-mt323:qt-mt323.dll
 0002:0000045c       __imp_?setNum@QLabel@@UAEXN@Z 1000445c     qt-mt323:qt-mt323.dll
 0002:00000460       __imp_?setOn@QPushButton@@UAEX_N@Z 10004460     qt-mt323:qt-mt323.dll
 0002:00000464       __imp_?setPicture@QLabel@@UAEXABVQPicture@@@Z 10004464     qt-mt323:qt-mt323.dll
 0002:00000468       __imp_?setPixmap@QButton@@UAEXABVQPixmap@@@Z 10004468     qt-mt323:qt-mt323.dll
 0002:0000046c       __imp_?setPixmap@QLabel@@UAEXABVQPixmap@@@Z 1000446c     qt-mt323:qt-mt323.dll
 0002:00000470       __imp_?setSpacing@QLayout@@UAEXH@Z 10004470     qt-mt323:qt-mt323.dll
 0002:00000474       __imp_?setState@QButton@@MAEXW4ToggleState@1@@Z 10004474     qt-mt323:qt-mt323.dll
 0002:00000478       __imp_?setText@QButton@@UAEXABVQString@@@Z 10004478     qt-mt323:qt-mt323.dll
 0002:0000047c       __imp_?setText@QLabel@@UAEXABVQString@@@Z 1000447c     qt-mt323:qt-mt323.dll
 0002:00000480       __imp_?setToggleType@QButton@@MAEXW4ToggleType@1@@Z 10004480     qt-mt323:qt-mt323.dll
 0002:00000484       __imp_?sizeHint@QBoxLayout@@UBE?AVQSize@@XZ 10004484     qt-mt323:qt-mt323.dll
 0002:00000488       __imp_?sizeHint@QLabel@@UBE?AVQSize@@XZ 10004488     qt-mt323:qt-mt323.dll
 0002:0000048c       __imp_?sizeHint@QPushButton@@UBE?AVQSize@@XZ 1000448c     qt-mt323:qt-mt323.dll
 0002:00000490       __imp_?sizeHint@QSpacerItem@@UBE?AVQSize@@XZ 10004490     qt-mt323:qt-mt323.dll
 0002:00000494       __imp_?sizeHint@QWidget@@UBE?AVQSize@@XZ 10004494     qt-mt323:qt-mt323.dll
 0002:00000498       __imp_?spacerItem@QLayoutItem@@UAEPAVQSpacerItem@@XZ 10004498     qt-mt323:qt-mt323.dll
 0002:0000049c       __imp_?spacerItem@QSpacerItem@@UAEPAV1@XZ 1000449c     qt-mt323:qt-mt323.dll
 0002:000004a0       __imp_?styleChange@QWidget@@MAEXAAVQStyle@@@Z 100044a0     qt-mt323:qt-mt323.dll
 0002:000004a4       __imp_?updateMask@QPushButton@@MAEXXZ 100044a4     qt-mt323:qt-mt323.dll
 0002:000004a8       __imp_?widget@QLayoutItem@@UAEPAVQWidget@@XZ 100044a8     qt-mt323:qt-mt323.dll
 0002:000004ac       __imp_?activate_signal@QObject@@IAEXHVQString@@@Z 100044ac     qt-mt323:qt-mt323.dll
 0002:000004b0       __imp_?qt_cast@QVBox@@UAEPAXPBD@Z 100044b0     qt-mt323:qt-mt323.dll
 0002:000004b4       __imp_?qt_invoke@QVBox@@UAE_NHPAUQUObject@@@Z 100044b4     qt-mt323:qt-mt323.dll
 0002:000004b8       __imp_?qt_emit@QVBox@@UAE_NHPAUQUObject@@@Z 100044b8     qt-mt323:qt-mt323.dll
 0002:000004bc       __imp_?qt_property@QVBox@@UAE_NHHPAVQVariant@@@Z 100044bc     qt-mt323:qt-mt323.dll
 0002:000004c0       __imp_?staticMetaObject@QVBox@@SAPAVQMetaObject@@XZ 100044c0     qt-mt323:qt-mt323.dll
 0002:000004c4       __imp_?static_QUType_QString@@3UQUType_QString@@A 100044c4     qt-mt323:qt-mt323.dll
 0002:000004c8       __imp_??0QStringList@@QAE@ABV0@@Z 100044c8     qt-mt323:qt-mt323.dll
 0002:000004cc       __imp_??0QStringList@@QAE@XZ 100044cc     qt-mt323:qt-mt323.dll
 0002:000004d0       __imp_?connect@QObject@@SA_NPBV1@PBD01@Z 100044d0     qt-mt323:qt-mt323.dll
 0002:000004d4       __imp_?contains@?$QValueList@VQString@@@@QBEIABVQString@@@Z 100044d4     qt-mt323:qt-mt323.dll
 0002:000004d8       __imp_?findIndex@?$QValueList@VQString@@@@QBEHABVQString@@@Z 100044d8     qt-mt323:qt-mt323.dll
 0002:000004dc       __imp_?prepend@?$QValueList@VQString@@@@QAE?AV?$QValueListIterator@VQString@@@@ABVQString@@@Z 100044dc     qt-mt323:qt-mt323.dll
 0002:000004e0       __imp_?append@?$QValueList@VQString@@@@QAE?AV?$QValueListIterator@VQString@@@@ABVQString@@@Z 100044e0     qt-mt323:qt-mt323.dll
 0002:000004e4       __imp_?clear@?$QValueList@VQString@@@@QAEXXZ 100044e4     qt-mt323:qt-mt323.dll
 0002:000004e8       __imp_?attribute@QDomElement@@QBE?AVQString@@ABV2@0@Z 100044e8     qt-mt323:qt-mt323.dll
 0002:000004ec       __imp_??1QDomElement@@UAE@XZ 100044ec     qt-mt323:qt-mt323.dll
 0002:000004f0       __imp_?setContent@QDomDocument@@QAE_NABVQString@@PAV2@PAH2@Z 100044f0     qt-mt323:qt-mt323.dll
 0002:000004f4       __imp_?documentElement@QDomDocument@@QBE?AVQDomElement@@XZ 100044f4     qt-mt323:qt-mt323.dll
 0002:000004f8       __imp_??1QDomDocument@@UAE@XZ 100044f8     qt-mt323:qt-mt323.dll
 0002:000004fc       __imp_??0QDomDocument@@QAE@ABVQString@@@Z 100044fc     qt-mt323:qt-mt323.dll
 0002:00000500       __imp_?toElement@QDomNode@@QAE?AVQDomElement@@XZ 10004500     qt-mt323:qt-mt323.dll
 0002:00000504       __imp_?isNull@QDomNode@@QBE_NXZ 10004504     qt-mt323:qt-mt323.dll
 0002:00000508       __imp_?nextSibling@QDomNode@@UBE?AV1@XZ 10004508     qt-mt323:qt-mt323.dll
 0002:0000050c       __imp_?firstChild@QDomNode@@UBE?AV1@XZ 1000450c     qt-mt323:qt-mt323.dll
 0002:00000510       __imp_??1QDomNode@@UAE@XZ  10004510     qt-mt323:qt-mt323.dll
 0002:00000514       __imp_??4QDomNode@@QAEAAV0@ABV0@@Z 10004514     qt-mt323:qt-mt323.dll
 0002:00000518       __imp_??H@YA?BVQString@@ABV0@0@Z 10004518     qt-mt323:qt-mt323.dll
 0002:0000051c       __imp_??H@YA?BVQString@@ABV0@PBD@Z 1000451c     qt-mt323:qt-mt323.dll
 0002:00000520       __imp_?makeSharedNull@QString@@CAPAUQStringData@@XZ 10004520     qt-mt323:qt-mt323.dll
 0002:00000524       __imp_?contains@QString@@QBEHPBD_N@Z 10004524     qt-mt323:qt-mt323.dll
 0002:00000528       __imp_??4QString@@QAEAAV0@PBD@Z 10004528     qt-mt323:qt-mt323.dll
 0002:0000052c       __imp_??4QString@@QAEAAV0@ABV0@@Z 1000452c     qt-mt323:qt-mt323.dll
 0002:00000530       __imp_??1QString@@QAE@XZ   10004530     qt-mt323:qt-mt323.dll
 0002:00000534       __imp_??0QString@@QAE@PBD@Z 10004534     qt-mt323:qt-mt323.dll
 0002:00000538       __imp_??0QString@@QAE@ABV0@@Z 10004538     qt-mt323:qt-mt323.dll
 0002:0000053c       __imp_?qApp@@3PAVQApplication@@A 1000453c     qt-mt323:qt-mt323.dll
 0002:00000540       __imp_?deleteSelf@QStringData@@QAEXXZ 10004540     qt-mt323:qt-mt323.dll
 0002:00000544       \177qt-mt323_NULL_THUNK_DATA 10004544     qt-mt323:qt-mt323.dll
 0002:00000548       ___xc_a                    10004548     MSVCRT:cinitexe.obj
 0002:00000558       ___xc_z                    10004558     MSVCRT:cinitexe.obj
 0002:0000055c       ___xi_a                    1000455c     MSVCRT:cinitexe.obj
 0002:00000568       ___xi_z                    10004568     MSVCRT:cinitexe.obj
 0002:00000574       ??_7CAlm_sys_select@@6BQObject@@@ 10004574     alm_sys_select.obj
 0002:00000748       ??_7CAlm_sys_select@@6BQPaintDevice@@@ 10004748     alm_sys_select.obj
 0002:00000768       ??_C@_0BJ@EFHKANIO@?$DMh2?$DOselect?5a?5system?$DM?1h2?$DO?$AA@ 10004768     alm_sys_select.obj
 0002:00000784       ??_C@_05OGKMNEDA@?$DM?1h2?$DO?$AA@ 10004784     alm_sys_select.obj
 0002:0000078c       ??_C@_04MFLEKIAK@?$DMh2?$DO?$AA@ 1000478c     alm_sys_select.obj
 0002:00000794       ??_C@_0BA@BODCLBBG@1selectSystem?$CI?$CJ?$AA@ 10004794     alm_sys_select.obj
 0002:000007a4       ??_C@_0M@PIBNEBIG@2released?$CI?$CJ?$AA@ 100047a4     alm_sys_select.obj
 0002:000007b0       ??_C@_05BHLILLHF@myDoc?$AA@ 100047b0     alm_sys_select.obj
 0002:000007b8       ??_C@_04JNIHBGGH@date?$AA@ 100047b8     alm_sys_select.obj
 0002:000007c0       ??_C@_04MEMAJGDJ@name?$AA@ 100047c0     alm_sys_select.obj
 0002:000007c8       ??_C@_01KMDKNFGN@?1?$AA@   100047c8     alm_sys_select.obj
 0002:000007ca       ??_C@_00CNPNBAHC@?$AA@     100047ca     alm_sys_select.obj
 0002:000007cc       ??_C@_0BE@HCIAKODO@Select?5Alarm?5System?$AA@ 100047cc     alm_sys_select.obj
 0002:000007e0       ??_C@_0BJ@MKHLJCJC@BNCS?5Alarm?5Configuration?$AA@ 100047e0     alm_sys_select.obj
 0002:000007fc       ??_C@_0P@IFMODJFN@sys_selectBase?$AA@ 100047fc     moc_sys_select.obj
 0002:00000818       ??_C@_0P@DMEOIADN@languageChange?$AA@ 10004818     moc_sys_select.obj
 0002:00000834       ??_C@_0BB@PFEIHPGD@languageChange?$CI?$CJ?$AA@ 10004834     moc_sys_select.obj
 0002:0000084c       ??_7sys_selectBase@@6BQObject@@@ 1000484c     sys_select.obj
 0002:00000a04       ??_7sys_selectBase@@6BQPaintDevice@@@ 10004a04     sys_select.obj
 0002:00000a2c       ??_SQPushButton@@6BQObject@@@ 10004a2c     sys_select.obj
 0002:00000c1c       ??_SQPushButton@@6BQPaintDevice@@@ 10004c1c     sys_select.obj
 0002:00000c44       ??_SQLabel@@6BQObject@@@   10004c44     sys_select.obj
 0002:00000e3c       ??_SQLabel@@6BQPaintDevice@@@ 10004e3c     sys_select.obj
 0002:00000e64       ??_SQSpacerItem@@6B@       10004e64     sys_select.obj
 0002:00000eac       ??_SQHBoxLayout@@6BQObject@@@ 10004eac     sys_select.obj
 0002:00000f14       ??_SQHBoxLayout@@6BQLayoutItem@@@ 10004f14     sys_select.obj
 0002:00000f5c       ??_SQVBoxLayout@@6BQObject@@@ 10004f5c     sys_select.obj
 0002:00000fc4       ??_SQVBoxLayout@@6BQLayoutItem@@@ 10004fc4     sys_select.obj
 0002:00001004       ??_C@_0BA@GBBFFEEM@sizeGripEnabled?$AA@ 10005004     sys_select.obj
 0002:00001014       ??_C@_0BF@KDKADBNA@sys_selectBaseLayout?$AA@ 10005014     sys_select.obj
 0002:0000102c       ??_C@_07OFHOKKPF@layout2?$AA@ 1000502c     sys_select.obj
 0002:00001034       ??_C@_0L@KGLFILOJ@textLabel1?$AA@ 10005034     sys_select.obj
 0002:00001040       ??_C@_0M@IGPKOKGF@labelSystem?$AA@ 10005040     sys_select.obj
 0002:0000104c       ??_C@_07PMGFJLLE@layout3?$AA@ 1000504c     sys_select.obj
 0002:00001054       ??_C@_0N@GONCKGLK@buttonChange?$AA@ 10005054     sys_select.obj
 0002:00001064       ??_C@_0L@GIINMKGA@sys_select?$AA@ 10005064     sys_select.obj
 0002:00001070       ??_C@_0P@MPFLAGHA@Current?5System?$AA@ 10005070     sys_select.obj
 0002:00001080       ??_C@_09BOCENGOA@?$DMh2?$DO?$DM?1h2?$DO?$AA@ 10005080     sys_select.obj
 0002:0000108c       ??_C@_0O@NAPAGHBK@Change?5System?$AA@ 1000508c     sys_select.obj
 0002:0000109c       ??_C@_0BA@DKBPLDBN@CAlm_sys_select?$AA@ 1000509c     moc_alm_sys_select.obj
 0002:000010b8       ??_C@_0N@JNMAEFDJ@selectSystem?$AA@ 100050b8     moc_alm_sys_select.obj
 0002:000010d4       ??_C@_0P@HKCKCNNG@selectSystem?$CI?$CJ?$AA@ 100050d4     moc_alm_sys_select.obj
 0002:000010f0       ??_C@_0L@CDFHJBCO@sysChanged?$AA@ 100050f0     moc_alm_sys_select.obj
 0002:00001108       ??_C@_0BL@HOJPHBGM@sysChanged?$CIconst?5QString?$CG?$CJ?$AA@ 10005108     moc_alm_sys_select.obj
 0002:00001128       ??_7type_info@@6B@         10005128     MSVCRT:ti_inst.obj
 0002:0000112c       __pDefaultRawDllMain       1000512c     MSVCRT:crtdll.obj
 0002:0000112c       __pRawDllMain              1000512c     MSVCRT:crtdll.obj
 0002:00001138       __load_config_used         10005138     MSVCRT:loadcfg.obj
 0002:00001180       ??_R1A@?0A@EA@QWidget@@8   10005180     alm_sys_select.obj
 0002:0000119c       ??_R3QWidget@@8            1000519c     alm_sys_select.obj
 0002:000011ac       ??_R2QWidget@@8            100051ac     alm_sys_select.obj
 0002:000011c0       ??_R1A@?0A@EA@QObject@@8   100051c0     alm_sys_select.obj
 0002:000011dc       ??_R3QObject@@8            100051dc     alm_sys_select.obj
 0002:000011ec       ??_R2QObject@@8            100051ec     alm_sys_select.obj
 0002:000011f8       ??_R13?0A@EA@Qt@@8         100051f8     alm_sys_select.obj
 0002:00001214       ??_R3Qt@@8                 10005214     alm_sys_select.obj
 0002:00001224       ??_R2Qt@@8                 10005224     alm_sys_select.obj
 0002:0000122c       ??_R1A@?0A@EA@Qt@@8        1000522c     alm_sys_select.obj
 0002:00001248       ??_R1CI@?0A@EA@QPaintDevice@@8 10005248     alm_sys_select.obj
 0002:00001264       ??_R3QPaintDevice@@8       10005264     alm_sys_select.obj
 0002:00001274       ??_R2QPaintDevice@@8       10005274     alm_sys_select.obj
 0002:0000127c       ??_R1A@?0A@EA@QPaintDevice@@8 1000527c     alm_sys_select.obj
 0002:00001298       ??_R4CAlm_sys_select@@6BQObject@@@ 10005298     alm_sys_select.obj
 0002:000012ac       ??_R3CAlm_sys_select@@8    100052ac     alm_sys_select.obj
 0002:000012bc       ??_R2CAlm_sys_select@@8    100052bc     alm_sys_select.obj
 0002:000012e0       ??_R1A@?0A@EA@CAlm_sys_select@@8 100052e0     alm_sys_select.obj
 0002:000012fc       ??_R1A@?0A@EA@QVBox@@8     100052fc     alm_sys_select.obj
 0002:00001318       ??_R3QVBox@@8              10005318     alm_sys_select.obj
 0002:00001328       ??_R2QVBox@@8              10005328     alm_sys_select.obj
 0002:00001348       ??_R1A@?0A@EA@QHBox@@8     10005348     alm_sys_select.obj
 0002:00001364       ??_R3QHBox@@8              10005364     alm_sys_select.obj
 0002:00001374       ??_R2QHBox@@8              10005374     alm_sys_select.obj
 0002:00001390       ??_R1A@?0A@EA@QFrame@@8    10005390     alm_sys_select.obj
 0002:000013ac       ??_R3QFrame@@8             100053ac     alm_sys_select.obj
 0002:000013bc       ??_R2QFrame@@8             100053bc     alm_sys_select.obj
 0002:000013d4       ??_R4CAlm_sys_select@@6BQPaintDevice@@@ 100053d4     alm_sys_select.obj
 0002:000013e8       ??_R4QVBoxLayout@@6BQObject@@@ 100053e8     sys_select.obj
 0002:000013fc       ??_R3QVBoxLayout@@8        100053fc     sys_select.obj
 0002:0000140c       ??_R2QVBoxLayout@@8        1000540c     sys_select.obj
 0002:00001428       ??_R1A@?0A@EA@QVBoxLayout@@8 10005428     sys_select.obj
 0002:00001444       ??_R1A@?0A@EA@QBoxLayout@@8 10005444     sys_select.obj
 0002:00001460       ??_R3QBoxLayout@@8         10005460     sys_select.obj
 0002:00001470       ??_R2QBoxLayout@@8         10005470     sys_select.obj
 0002:00001488       ??_R1A@?0A@EA@QLayout@@8   10005488     sys_select.obj
 0002:000014a4       ??_R3QLayout@@8            100054a4     sys_select.obj
 0002:000014b4       ??_R2QLayout@@8            100054b4     sys_select.obj
 0002:000014c8       ??_R1CI@?0A@EA@QLayoutItem@@8 100054c8     sys_select.obj
 0002:000014e4       ??_R3QLayoutItem@@8        100054e4     sys_select.obj
 0002:000014f4       ??_R2QLayoutItem@@8        100054f4     sys_select.obj
 0002:000014fc       ??_R1A@?0A@EA@QLayoutItem@@8 100054fc     sys_select.obj
 0002:00001518       ??_R4QVBoxLayout@@6BQLayoutItem@@@ 10005518     sys_select.obj
 0002:0000152c       ??_R4QHBoxLayout@@6BQObject@@@ 1000552c     sys_select.obj
 0002:00001540       ??_R3QHBoxLayout@@8        10005540     sys_select.obj
 0002:00001550       ??_R2QHBoxLayout@@8        10005550     sys_select.obj
 0002:0000156c       ??_R1A@?0A@EA@QHBoxLayout@@8 1000556c     sys_select.obj
 0002:00001588       ??_R4QHBoxLayout@@6BQLayoutItem@@@ 10005588     sys_select.obj
 0002:0000159c       ??_R4QLabel@@6BQObject@@@  1000559c     sys_select.obj
 0002:000015b0       ??_R3QLabel@@8             100055b0     sys_select.obj
 0002:000015c0       ??_R2QLabel@@8             100055c0     sys_select.obj
 0002:000015dc       ??_R1A@?0A@EA@QLabel@@8    100055dc     sys_select.obj
 0002:000015f8       ??_R4QLabel@@6BQPaintDevice@@@ 100055f8     sys_select.obj
 0002:0000160c       ??_R4QPushButton@@6BQObject@@@ 1000560c     sys_select.obj
 0002:00001620       ??_R3QPushButton@@8        10005620     sys_select.obj
 0002:00001630       ??_R2QPushButton@@8        10005630     sys_select.obj
 0002:0000164c       ??_R1A@?0A@EA@QPushButton@@8 1000564c     sys_select.obj
 0002:00001668       ??_R1A@?0A@EA@QButton@@8   10005668     sys_select.obj
 0002:00001684       ??_R3QButton@@8            10005684     sys_select.obj
 0002:00001694       ??_R2QButton@@8            10005694     sys_select.obj
 0002:000016ac       ??_R4QPushButton@@6BQPaintDevice@@@ 100056ac     sys_select.obj
 0002:000016c0       ??_R4sys_selectBase@@6BQObject@@@ 100056c0     sys_select.obj
 0002:000016d4       ??_R3sys_selectBase@@8     100056d4     sys_select.obj
 0002:000016e4       ??_R2sys_selectBase@@8     100056e4     sys_select.obj
 0002:000016fc       ??_R1A@?0A@EA@sys_selectBase@@8 100056fc     sys_select.obj
 0002:00001718       ??_R4sys_selectBase@@6BQPaintDevice@@@ 10005718     sys_select.obj
 0002:0000172c       ??_R4QSpacerItem@@6B@      1000572c     sys_select.obj
 0002:00001740       ??_R3QSpacerItem@@8        10005740     sys_select.obj
 0002:00001750       ??_R2QSpacerItem@@8        10005750     sys_select.obj
 0002:0000175c       ??_R1A@?0A@EA@QSpacerItem@@8 1000575c     sys_select.obj
 0002:00001778       ??_R4type_info@@6B@        10005778     MSVCRT:ti_inst.obj
 0002:0000178c       ??_R3type_info@@8          1000578c     MSVCRT:ti_inst.obj
 0002:0000179c       ??_R2type_info@@8          1000579c     MSVCRT:ti_inst.obj
 0002:000017a4       ??_R1A@?0A@EA@type_info@@8 100057a4     MSVCRT:ti_inst.obj
 0002:000017c0       ___rtc_iaa                 100057c0     MSVCRT:initsect.obj
 0002:000017c4       ___rtc_izz                 100057c4     MSVCRT:initsect.obj
 0002:000017c8       ___rtc_taa                 100057c8     MSVCRT:initsect.obj
 0002:000017cc       ___rtc_tzz                 100057cc     MSVCRT:initsect.obj
 0002:000020e0       __IMPORT_DESCRIPTOR_qt-mt323 100060e0     qt-mt323:qt-mt323.dll
 0002:000020f4       __IMPORT_DESCRIPTOR_MSVCR120 100060f4     MSVCRT:MSVCR120.dll
 0002:00002108       __IMPORT_DESCRIPTOR_KERNEL32 10006108     kernel32:KERNEL32.dll
 0002:0000211c       __NULL_IMPORT_DESCRIPTOR   1000611c     qt-mt323:qt-mt323.dll
 0003:00000000       ___security_cookie         1000a000     MSVCRT:gs_cookie.obj
 0003:00000004       ___security_cookie_complement 1000a004     MSVCRT:gs_cookie.obj
 0003:00000010       ___native_dllmain_reason   1000a010     MSVCRT:natstart.obj
 0003:00000014       ??_R0?AVQWidget@@@8        1000a014     alm_sys_select.obj
 0003:0000002c       ??_R0?AVQObject@@@8        1000a02c     alm_sys_select.obj
 0003:00000044       ??_R0?AVQt@@@8             1000a044     alm_sys_select.obj
 0003:00000058       ??_R0?AVQPaintDevice@@@8   1000a058     alm_sys_select.obj
 0003:00000074       ??_R0?AVCAlm_sys_select@@@8 1000a074     alm_sys_select.obj
 0003:00000094       ??_R0?AVQVBox@@@8          1000a094     alm_sys_select.obj
 0003:000000a8       ??_R0?AVQHBox@@@8          1000a0a8     alm_sys_select.obj
 0003:000000bc       ??_R0?AVQFrame@@@8         1000a0bc     alm_sys_select.obj
 0003:000000d4       ??_R0?AVQVBoxLayout@@@8    1000a0d4     sys_select.obj
 0003:000000f0       ??_R0?AVQBoxLayout@@@8     1000a0f0     sys_select.obj
 0003:0000010c       ??_R0?AVQLayout@@@8        1000a10c     sys_select.obj
 0003:00000124       ??_R0?AVQLayoutItem@@@8    1000a124     sys_select.obj
 0003:00000140       ??_R0?AVQHBoxLayout@@@8    1000a140     sys_select.obj
 0003:0000015c       ??_R0?AVQLabel@@@8         1000a15c     sys_select.obj
 0003:00000174       ??_R0?AVQPushButton@@@8    1000a174     sys_select.obj
 0003:00000190       ??_R0?AVQButton@@@8        1000a190     sys_select.obj
 0003:000001a8       ??_R0?AVsys_selectBase@@@8 1000a1a8     sys_select.obj
 0003:000001c8       ??_R0?AVQSpacerItem@@@8    1000a1c8     sys_select.obj
 0003:000001e4       ??_R0?AVtype_info@@@8      1000a1e4     MSVCRT:ti_inst.obj
 0003:00000200       ?sCurrentSystem@CAlm_sys_select@@0VQString@@A 1000a200     alm_sys_select.obj
 0003:00000204       ?metaObj@sys_selectBase@@0PAVQMetaObject@@A 1000a204     moc_sys_select.obj
 0003:0000020c       ?metaObj@CAlm_sys_select@@0PAVQMetaObject@@A 1000a20c     moc_alm_sys_select.obj
 0003:00000550       ?__type_info_root_node@@3U__type_info_node@@A 1000a550     MSVCRT:tncleanup.obj
 0003:00000558       ___native_startup_lock     1000a558     <common>
 0003:0000055c       ___native_startup_state    1000a55c     <common>
 0003:00000560       ___dyn_tls_init_callback   1000a560     <common>
 0003:00000564       ___onexitend               1000a564     <common>
 0003:00000568       ___onexitbegin             1000a568     <common>

 entry point at        0001:00001e71

 Static symbols

 0001:00000000       ??__E?sCurrentSystem@CAlm_sys_select@@0VQString@@A@@YAXXZ 10001000 f   alm_sys_select.obj
 0001:00000030       ??__EcleanUp_sys_selectBase@@YAXXZ 10001030 f   moc_sys_select.obj
 0001:00000060       ??__EcleanUp_CAlm_sys_select@@YAXXZ 10001060 f   moc_alm_sys_select.obj
 0001:00001c2e       _pre_c_init                10002c2e f   MSVCRT:crtdll.obj
 0001:00001e94       ___DllMainCRTStartup       10002e94 f   MSVCRT:crtdll.obj
 0001:00001fd0       $$000000                   10002fd0     MSVCRT:sehprolg4.obj
 0001:00002410       __unwindfunclet$??0CAlm_sys_select@@QAE@PAVQWidget@@PBD@Z$0 10003410 f   alm_sys_select.obj
 0001:00002419       __unwindfunclet$??0CAlm_sys_select@@QAE@PAVQWidget@@PBD@Z$1 10003419 f   alm_sys_select.obj
 0001:00002428       __unwindfunclet$??0CAlm_sys_select@@QAE@PAVQWidget@@PBD@Z$2 10003428 f   alm_sys_select.obj
 0001:00002433       __unwindfunclet$??0CAlm_sys_select@@QAE@PAVQWidget@@PBD@Z$3 10003433 f   alm_sys_select.obj
 0001:0000243c       __unwindfunclet$??0CAlm_sys_select@@QAE@PAVQWidget@@PBD@Z$4 1000343c f   alm_sys_select.obj
 0001:00002445       __unwindfunclet$??0CAlm_sys_select@@QAE@PAVQWidget@@PBD@Z$5 10003445 f   alm_sys_select.obj
 0001:0000244e       __unwindfunclet$??0CAlm_sys_select@@QAE@PAVQWidget@@PBD@Z$6 1000344e f   alm_sys_select.obj
 0001:00002457       __ehhandler$??0CAlm_sys_select@@QAE@PAVQWidget@@PBD@Z 10003457 f   alm_sys_select.obj
 0001:00002480       __unwindfunclet$??1CAlm_sys_select@@UAE@XZ$0 10003480 f   alm_sys_select.obj
 0001:00002489       __ehhandler$??1CAlm_sys_select@@UAE@XZ 10003489 f   alm_sys_select.obj
 0001:000024b0       __unwindfunclet$??_ECAlm_sys_select@@UAEPAXI@Z$0 100034b0 f   alm_sys_select.obj
 0001:000024b9       __ehhandler$??_ECAlm_sys_select@@UAEPAXI@Z 100034b9 f   alm_sys_select.obj
 0001:000024e0       __unwindfunclet$?getSystemName@CAlm_sys_select@@QAE?AVQString@@XZ$0 100034e0 f   alm_sys_select.obj
 0001:000024e9       __unwindfunclet$?getSystemName@CAlm_sys_select@@QAE?AVQString@@XZ$1 100034e9 f   alm_sys_select.obj
 0001:000024f2       __unwindfunclet$?getSystemName@CAlm_sys_select@@QAE?AVQString@@XZ$2 100034f2 f   alm_sys_select.obj
 0001:000024fb       __unwindfunclet$?getSystemName@CAlm_sys_select@@QAE?AVQString@@XZ$3 100034fb f   alm_sys_select.obj
 0001:00002504       __ehhandler$?getSystemName@CAlm_sys_select@@QAE?AVQString@@XZ 10003504 f   alm_sys_select.obj
 0001:00002520       __unwindfunclet$?selectSystem@CAlm_sys_select@@IAEXXZ$0 10003520 f   alm_sys_select.obj
 0001:00002529       __unwindfunclet$?selectSystem@CAlm_sys_select@@IAEXXZ$1 10003529 f   alm_sys_select.obj
 0001:00002532       __unwindfunclet$?selectSystem@CAlm_sys_select@@IAEXXZ$2 10003532 f   alm_sys_select.obj
 0001:0000253b       __unwindfunclet$?selectSystem@CAlm_sys_select@@IAEXXZ$3 1000353b f   alm_sys_select.obj
 0001:00002544       __unwindfunclet$?selectSystem@CAlm_sys_select@@IAEXXZ$4 10003544 f   alm_sys_select.obj
 0001:0000254d       __unwindfunclet$?selectSystem@CAlm_sys_select@@IAEXXZ$5 1000354d f   alm_sys_select.obj
 0001:00002556       __unwindfunclet$?selectSystem@CAlm_sys_select@@IAEXXZ$6 10003556 f   alm_sys_select.obj
 0001:0000255f       __unwindfunclet$?selectSystem@CAlm_sys_select@@IAEXXZ$7 1000355f f   alm_sys_select.obj
 0001:00002568       __unwindfunclet$?selectSystem@CAlm_sys_select@@IAEXXZ$8 10003568 f   alm_sys_select.obj
 0001:00002571       __ehhandler$?selectSystem@CAlm_sys_select@@IAEXXZ 10003571 f   alm_sys_select.obj
 0001:00002590       __unwindfunclet$?setSystemNames@CAlm_sys_select@@QAE_NVQString@@@Z$0 10003590 f   alm_sys_select.obj
 0001:00002599       __unwindfunclet$?setSystemNames@CAlm_sys_select@@QAE_NVQString@@@Z$1 10003599 f   alm_sys_select.obj
 0001:000025a2       __unwindfunclet$?setSystemNames@CAlm_sys_select@@QAE_NVQString@@@Z$2 100035a2 f   alm_sys_select.obj
 0001:000025ab       __unwindfunclet$?setSystemNames@CAlm_sys_select@@QAE_NVQString@@@Z$3 100035ab f   alm_sys_select.obj
 0001:000025b4       __unwindfunclet$?setSystemNames@CAlm_sys_select@@QAE_NVQString@@@Z$4 100035b4 f   alm_sys_select.obj
 0001:000025bd       __unwindfunclet$?setSystemNames@CAlm_sys_select@@QAE_NVQString@@@Z$6 100035bd f   alm_sys_select.obj
 0001:000025c6       __unwindfunclet$?setSystemNames@CAlm_sys_select@@QAE_NVQString@@@Z$7 100035c6 f   alm_sys_select.obj
 0001:000025cf       __unwindfunclet$?setSystemNames@CAlm_sys_select@@QAE_NVQString@@@Z$8 100035cf f   alm_sys_select.obj
 0001:000025d8       __unwindfunclet$?setSystemNames@CAlm_sys_select@@QAE_NVQString@@@Z$9 100035d8 f   alm_sys_select.obj
 0001:000025e1       __unwindfunclet$?setSystemNames@CAlm_sys_select@@QAE_NVQString@@@Z$10 100035e1 f   alm_sys_select.obj
 0001:000025ea       __unwindfunclet$?setSystemNames@CAlm_sys_select@@QAE_NVQString@@@Z$5 100035ea f   alm_sys_select.obj
 0001:000025f3       __unwindfunclet$?setSystemNames@CAlm_sys_select@@QAE_NVQString@@@Z$11 100035f3 f   alm_sys_select.obj
 0001:000025fc       __unwindfunclet$?setSystemNames@CAlm_sys_select@@QAE_NVQString@@@Z$12 100035fc f   alm_sys_select.obj
 0001:00002605       __unwindfunclet$?setSystemNames@CAlm_sys_select@@QAE_NVQString@@@Z$13 10003605 f   alm_sys_select.obj
 0001:0000260e       __unwindfunclet$?setSystemNames@CAlm_sys_select@@QAE_NVQString@@@Z$14 1000360e f   alm_sys_select.obj
 0001:00002617       __unwindfunclet$?setSystemNames@CAlm_sys_select@@QAE_NVQString@@@Z$15 10003617 f   alm_sys_select.obj
 0001:00002620       __ehhandler$?setSystemNames@CAlm_sys_select@@QAE_NVQString@@@Z 10003620 f   alm_sys_select.obj
 0001:00002640       __unwindfunclet$??0sys_selectBase@@QAE@PAVQWidget@@PBDI@Z$0 10003640 f   sys_select.obj
 0001:00002649       __unwindfunclet$??0sys_selectBase@@QAE@PAVQWidget@@PBDI@Z$1 10003649 f   sys_select.obj
 0001:00002652       __unwindfunclet$??0sys_selectBase@@QAE@PAVQWidget@@PBDI@Z$2 10003652 f   sys_select.obj
 0001:0000265d       __unwindfunclet$??0sys_selectBase@@QAE@PAVQWidget@@PBDI@Z$3 1000365d f   sys_select.obj
 0001:00002668       __unwindfunclet$??0sys_selectBase@@QAE@PAVQWidget@@PBDI@Z$4 10003668 f   sys_select.obj
 0001:00002673       __unwindfunclet$??0sys_selectBase@@QAE@PAVQWidget@@PBDI@Z$5 10003673 f   sys_select.obj
 0001:0000267e       __unwindfunclet$??0sys_selectBase@@QAE@PAVQWidget@@PBDI@Z$6 1000367e f   sys_select.obj
 0001:00002689       __unwindfunclet$??0sys_selectBase@@QAE@PAVQWidget@@PBDI@Z$7 10003689 f   sys_select.obj
 0001:00002694       __ehhandler$??0sys_selectBase@@QAE@PAVQWidget@@PBDI@Z 10003694 f   sys_select.obj
 0001:000026b0       __unwindfunclet$?languageChange@sys_selectBase@@MAEXXZ$0 100036b0 f   sys_select.obj
 0001:000026b9       __unwindfunclet$?languageChange@sys_selectBase@@MAEXXZ$1 100036b9 f   sys_select.obj
 0001:000026c2       __unwindfunclet$?languageChange@sys_selectBase@@MAEXXZ$2 100036c2 f   sys_select.obj
 0001:000026cb       __unwindfunclet$?languageChange@sys_selectBase@@MAEXXZ$3 100036cb f   sys_select.obj
 0001:000026d4       __ehhandler$?languageChange@sys_selectBase@@MAEXXZ 100036d4 f   sys_select.obj
 0001:000026f0       __unwindfunclet$?qt_emit@CAlm_sys_select@@UAE_NHPAUQUObject@@@Z$0 100036f0 f   moc_alm_sys_select.obj
 0001:000026f9       __ehhandler$?qt_emit@CAlm_sys_select@@UAE_NHPAUQUObject@@@Z 100036f9 f   moc_alm_sys_select.obj
 0001:00002720       __unwindfunclet$?sysChanged@CAlm_sys_select@@IAEXABVQString@@@Z$0 10003720 f   moc_alm_sys_select.obj
 0001:00002729       __ehhandler$?sysChanged@CAlm_sys_select@@IAEXABVQString@@@Z 10003729 f   moc_alm_sys_select.obj
 0001:00002750       ??__F?sCurrentSystem@CAlm_sys_select@@0VQString@@A@@YAXXZ 10003750 f   alm_sys_select.obj
 0001:00002770       ??__FcleanUp_sys_selectBase@@YAXXZ 10003770 f   moc_sys_select.obj
 0001:00002780       ??__FcleanUp_CAlm_sys_select@@YAXXZ 10003780 f   moc_alm_sys_select.obj
 0002:0000054c       ?sCurrentSystem$initializer$@CAlm_sys_select@@0P6AXXZA 1000454c     alm_sys_select.obj
 0002:00000550       _cleanUp_sys_selectBase$initializer$ 10004550     moc_sys_select.obj
 0002:00000554       _cleanUp_CAlm_sys_select$initializer$ 10004554     moc_alm_sys_select.obj
 0002:00000560       _pcinit                    10004560     MSVCRT:crtdll.obj
 0002:00000564       _pinit                     10004564     MSVCRT:atonexit.obj
 0002:0000080c       ?slot_0@?3??staticMetaObject@sys_selectBase@@SAPAVQMetaObject@@XZ@4UQUMethod@@B 1000480c     moc_sys_select.obj
 0002:00000828       ?slot_tbl@?3??staticMetaObject@sys_selectBase@@SAPAVQMetaObject@@XZ@4QBUQMetaData@@B 10004828     moc_sys_select.obj
 0002:000010ac       ?slot_0@?3??staticMetaObject@CAlm_sys_select@@SAPAVQMetaObject@@XZ@4UQUMethod@@B 100050ac     moc_alm_sys_select.obj
 0002:000010c8       ?slot_tbl@?3??staticMetaObject@CAlm_sys_select@@SAPAVQMetaObject@@XZ@4QBUQMetaData@@B 100050c8     moc_alm_sys_select.obj
 0002:000010e4       ?signal_0@?3??staticMetaObject@CAlm_sys_select@@SAPAVQMetaObject@@XZ@4UQUMethod@@B 100050e4     moc_alm_sys_select.obj
 0002:000010fc       ?signal_tbl@?3??staticMetaObject@CAlm_sys_select@@SAPAVQMetaObject@@XZ@4QBUQMetaData@@B 100050fc     moc_alm_sys_select.obj
 0002:00001130       _GS_ExceptionPointers      10005130     MSVCRT:gs_report.obj
 0002:000017d0       __ehfuncinfo$??0CAlm_sys_select@@QAE@PAVQWidget@@PBD@Z 100057d0     alm_sys_select.obj
 0002:000017f4       __unwindtable$??0CAlm_sys_select@@QAE@PAVQWidget@@PBD@Z 100057f4     alm_sys_select.obj
 0002:0000182c       __unwindtable$?getSystemName@CAlm_sys_select@@QAE?AVQString@@XZ 1000582c     alm_sys_select.obj
 0002:0000184c       __ehfuncinfo$?getSystemName@CAlm_sys_select@@QAE?AVQString@@XZ 1000584c     alm_sys_select.obj
 0002:00001870       __ehfuncinfo$?setSystemNames@CAlm_sys_select@@QAE_NVQString@@@Z 10005870     alm_sys_select.obj
 0002:00001894       __unwindtable$?setSystemNames@CAlm_sys_select@@QAE_NVQString@@@Z 10005894     alm_sys_select.obj
 0002:0000192c       __ehfuncinfo$?selectSystem@CAlm_sys_select@@IAEXXZ 1000592c     alm_sys_select.obj
 0002:00001950       __unwindtable$?selectSystem@CAlm_sys_select@@IAEXXZ 10005950     alm_sys_select.obj
 0002:000019a8       __unwindtable$??1CAlm_sys_select@@UAE@XZ 100059a8     alm_sys_select.obj
 0002:000019b0       __ehfuncinfo$??1CAlm_sys_select@@UAE@XZ 100059b0     alm_sys_select.obj
 0002:000019d4       __unwindtable$??_ECAlm_sys_select@@UAEPAXI@Z 100059d4     alm_sys_select.obj
 0002:000019dc       __ehfuncinfo$??_ECAlm_sys_select@@UAEPAXI@Z 100059dc     alm_sys_select.obj
 0002:00001a00       __ehfuncinfo$??0sys_selectBase@@QAE@PAVQWidget@@PBDI@Z 10005a00     sys_select.obj
 0002:00001a24       __unwindtable$??0sys_selectBase@@QAE@PAVQWidget@@PBDI@Z 10005a24     sys_select.obj
 0002:00001a64       __unwindtable$?languageChange@sys_selectBase@@MAEXXZ 10005a64     sys_select.obj
 0002:00001a84       __ehfuncinfo$?languageChange@sys_selectBase@@MAEXXZ 10005a84     sys_select.obj
 0002:00001aa8       __unwindtable$?qt_emit@CAlm_sys_select@@UAE_NHPAUQUObject@@@Z 10005aa8     moc_alm_sys_select.obj
 0002:00001ab0       __ehfuncinfo$?qt_emit@CAlm_sys_select@@UAE_NHPAUQUObject@@@Z 10005ab0     moc_alm_sys_select.obj
 0002:00001ad4       __unwindtable$?sysChanged@CAlm_sys_select@@IAEXABVQString@@@Z 10005ad4     moc_alm_sys_select.obj
 0002:00001adc       __ehfuncinfo$?sysChanged@CAlm_sys_select@@IAEXABVQString@@@Z 10005adc     moc_alm_sys_select.obj
 0002:00001b00       __sehtable$??_M@YGXPAXIHP6EX0@Z@Z 10005b00     MSVCRT:ehvecdtr.obj
 0002:00001b20       __sehtable$?__ArrayUnwind@@YGXPAXIHP6EX0@Z@Z 10005b20     MSVCRT:ehvecdtr.obj
 0002:00001b40       __sehtable$__onexit        10005b40     MSVCRT:atonexit.obj
 0002:00001b60       __sehtable$___DllMainCRTStartup 10005b60     MSVCRT:crtdll.obj
 0002:00001b88       __sehtable$__IsNonwritableInCurrentImage 10005b88     MSVCRT:pesect.obj
 0002:00001bb0       .edata                     10005bb0     alm_sys_select.exp
 0002:00001bd8       rgpv                       10005bd8     alm_sys_select.exp
 0002:00001c34       rgszName                   10005c34     alm_sys_select.exp
 0002:00001c90       rgwOrd                     10005c90     alm_sys_select.exp
 0002:00001cbe       szName                     10005cbe     alm_sys_select.exp
 0002:00001cd1       $N00001                    10005cd1     alm_sys_select.exp
 0002:00001cfb       $N00002                    10005cfb     alm_sys_select.exp
 0002:00001d16       $N00003                    10005d16     alm_sys_select.exp
 0002:00001d3a       $N00004                    10005d3a     alm_sys_select.exp
 0002:00001d5c       $N00005                    10005d5c     alm_sys_select.exp
 0002:00001d83       $N00006                    10005d83     alm_sys_select.exp
 0002:00001da8       $N00007                    10005da8     alm_sys_select.exp
 0002:00001dda       $N00008                    10005dda     alm_sys_select.exp
 0002:00001e07       $N00009                    10005e07     alm_sys_select.exp
 0002:00001e3a       $N00010                    10005e3a     alm_sys_select.exp
 0002:00001e66       $N00011                    10005e66     alm_sys_select.exp
 0002:00001e8c       $N00012                    10005e8c     alm_sys_select.exp
 0002:00001ebc       $N00013                    10005ebc     alm_sys_select.exp
 0002:00001eee       $N00014                    10005eee     alm_sys_select.exp
 0002:00001f23       $N00015                    10005f23     alm_sys_select.exp
 0002:00001f6a       $N00016                    10005f6a     alm_sys_select.exp
 0002:00001f98       $N00017                    10005f98     alm_sys_select.exp
 0002:00001fbe       $N00018                    10005fbe     alm_sys_select.exp
 0002:00001fed       $N00019                    10005fed     alm_sys_select.exp
 0002:00002020       $N00020                    10006020     alm_sys_select.exp
 0002:00002058       $N00021                    10006058     alm_sys_select.exp
 0002:00002088       $N00022                    10006088     alm_sys_select.exp
 0002:000020b2       $N00023                    100060b2     alm_sys_select.exp
 0002:000057b6       .idata$6                   100097b6     qt-mt323:qt-mt323.dll
 0002:0000580e       .idata$6                   1000980e     MSVCRT:MSVCR120.dll
 0002:000059f2       .idata$6                   100099f2     kernel32:KERNEL32.dll
 0003:00000208       _cleanUp_sys_selectBase    1000a208     moc_sys_select.obj
 0003:00000210       _cleanUp_CAlm_sys_select   1000a210     moc_alm_sys_select.obj
 0003:00000214       ?param_signal_0@?3??staticMetaObject@CAlm_sys_select@@SAPAVQMetaObject@@XZ@4QBUQUParameter@@B 1000a214     moc_alm_sys_select.obj
 0003:00000224       ?$S1@?3??staticMetaObject@CAlm_sys_select@@SAPAVQMetaObject@@XZ@4IA 1000a224     moc_alm_sys_select.obj
 0003:00000228       ___proc_attached           1000a228     MSVCRT:crtdll.obj
 0003:00000230       _GS_ExceptionRecord        1000a230     MSVCRT:gs_report.obj
 0003:00000280       _GS_ContextRecord          1000a280     MSVCRT:gs_report.obj
 0003:0000054c       _DebuggerWasPresent        1000a54c     MSVCRT:gs_report.obj
 0004:000000a0       $R000000                   1000b0a0     version.res
 0004:00000540       $R0004A0                   1000b540     version.res

 Exports

  ordinal    name

        1    ??0CAlm_sys_select@@QAE@PAVQWidget@@PBD@Z (public: __thiscall CAlm_sys_select::CAlm_sys_select(class QWidget *,char const *))
        2    ??1CAlm_sys_select@@UAE@XZ (public: virtual __thiscall CAlm_sys_select::~CAlm_sys_select(void))
        3    ??4CAlm_sys_select@@QAEAAV0@ABV0@@Z (public: class CAlm_sys_select & __thiscall CAlm_sys_select::operator=(class CAlm_sys_select const &))
        4    ??_7CAlm_sys_select@@6BQObject@@@ (const CAlm_sys_select::`vftable'{for `QObject'})
        5    ??_7CAlm_sys_select@@6BQPaintDevice@@@ (const CAlm_sys_select::`vftable'{for `QPaintDevice'})
        6    ?className@CAlm_sys_select@@UBEPBDXZ (public: virtual char const * __thiscall CAlm_sys_select::className(void)const )
        7    ?getSystemName@CAlm_sys_select@@QAE?AVQString@@XZ (public: class QString __thiscall CAlm_sys_select::getSystemName(void))
        8    ?metaObj@CAlm_sys_select@@0PAVQMetaObject@@A (private: static class QMetaObject * CAlm_sys_select::metaObj)
        9    ?metaObject@CAlm_sys_select@@UBEPAVQMetaObject@@XZ (public: virtual class QMetaObject * __thiscall CAlm_sys_select::metaObject(void)const )
       10    ?qObject@CAlm_sys_select@@QAEPAVQObject@@XZ (public: class QObject * __thiscall CAlm_sys_select::qObject(void))
       11    ?qt_cast@CAlm_sys_select@@UAEPAXPBD@Z (public: virtual void * __thiscall CAlm_sys_select::qt_cast(char const *))
       12    ?qt_emit@CAlm_sys_select@@UAE_NHPAUQUObject@@@Z (public: virtual bool __thiscall CAlm_sys_select::qt_emit(int,struct QUObject *))
       13    ?qt_invoke@CAlm_sys_select@@UAE_NHPAUQUObject@@@Z (public: virtual bool __thiscall CAlm_sys_select::qt_invoke(int,struct QUObject *))
       14    ?qt_property@CAlm_sys_select@@UAE_NHHPAVQVariant@@@Z (public: virtual bool __thiscall CAlm_sys_select::qt_property(int,int,class QVariant *))
       15    ?qt_static_property@CAlm_sys_select@@SA_NPAVQObject@@HHPAVQVariant@@@Z (public: static bool __cdecl CAlm_sys_select::qt_static_property(class QObject *,int,int,class QVariant *))
       16    ?sCurrentSystem@CAlm_sys_select@@0VQString@@A (private: static class QString CAlm_sys_select::sCurrentSystem)
       17    ?selectSystem@CAlm_sys_select@@IAEXXZ (protected: void __thiscall CAlm_sys_select::selectSystem(void))
       18    ?setSystem@CAlm_sys_select@@QAEXABVQString@@@Z (public: void __thiscall CAlm_sys_select::setSystem(class QString const &))
       19    ?setSystemNames@CAlm_sys_select@@QAE_NVQString@@@Z (public: bool __thiscall CAlm_sys_select::setSystemNames(class QString))
       20    ?staticMetaObject@CAlm_sys_select@@SAPAVQMetaObject@@XZ (public: static class QMetaObject * __cdecl CAlm_sys_select::staticMetaObject(void))
       21    ?sysChanged@CAlm_sys_select@@IAEXABVQString@@@Z (protected: void __thiscall CAlm_sys_select::sysChanged(class QString const &))
       22    ?tr@CAlm_sys_select@@SA?AVQString@@PBD0@Z (public: static class QString __cdecl CAlm_sys_select::tr(char const *,char const *))
       23    ?trUtf8@CAlm_sys_select@@SA?AVQString@@PBD0@Z (public: static class QString __cdecl CAlm_sys_select::trUtf8(char const *,char const *))
